:10673900202020202020202020200025622A626499
:106749000025622A62750025622A640025622A757D
:106759000025622A2E622A660025622A6C640025B9
:10676900622A6C7500253262753A25730020202053
:106779002020202020004E6F207661726961626CB2
:10678900657320646566696E656400202020202099
:1067990020202020202020202020202020200045EB
:1067A900534320454E5445522020202D202020209F
:1067B9002B20200045534320454E5445522020208C
:1067C9002D20202020202B200045534320454E54C6
:1067D90045522020200045534320202020202020FE
:1067E9002020002020202020002000506172616DAF
:1067F9006574657273207772697474656E00746F5D
:1068090020666C617368206D656D6F72792E00F476
:1068190070000000F76E000000FA8F000000FD6DA7
:106829000000000000000000036B000000064D009E
:10683900000009470000000C54000000630000003C
:1068490000016D00000002670000000373000000F2
:10685900046D000000056800000006410000000703
:106869004B000000088043000009804600001448DE
:106879007A00001550610000166261000017570088
:106889000000185600000019B50000001A54000055
:10689900001B6C2F73001C52504D001D4600000058
:1068A9001E4A0000005A250000005B52504D005C52
:1068B900636E74005D78000000000000000002357E
:1068C9000000004E6F64652041647200008D010074
:1068D900000000000000003F8000000000000235B9
:1068E900000000477270204164720000008F0100AF
:1068F900000000000000003F8000000000000A388E
:1069090000000054696D650000000001097E010066
:10691900000000000000003F8000000000000A386D
:10692900000000446174650000000001096E010067
:10693900000000000000003F800000000000040883
:1069490000000154656D7000000000010946020055
:10695900000000000000003F800000000000041853
:10696900000001312E38560000000001095E0200C6
:1069790000000000000000400000000000000418B2
:10698900000001332E33560000000001094A0200BD
:106999000000000000000040000000000000041892
:1069A90000000135566578740000000109520200A3
:1069B9000000000000000040000000000000041872
:1069C900000001323456000000000001095602009F
:1069D900000000000000003F8000000000000418D3
:1069E900000001323456657874000001095A02002A
:1069F900000000000000003F8000000000000406C5
:106A0900000001492032345600000001094E0200FD
:106A190000000000000000400000000000000032FB
:106A2900000004466C61736800000000000000006B
:106A3900000000000000000000000000000000321B
:106A49000000045265626F6F7400000000000000CE
:0E6A590000000000000000000000000000002F
:0AADBF00C19FC127C126C120C12198
:066A67008B3F8A408941CB
:106A6D0090000112072164387060854248854349C2
:106A7D0085444AF54B754C0A7B017A09796212AB54
:106A8D00DF7B017A09796212000EC3EF940AEE647E
:106A9D008094805032E490099BF07B017A097962F1
:106AAD0012000EC3740A9FFFE49EFE90099BE0C383
:106ABD009FEE6480F8748098500D7F2012B326905D
:106ACD00099BE004F080D3026D2EE4900962F0ABD7
:106ADD003FAA40A9419000021207216068E4900985
:106AED009BF090099BE075F005A42418F582E43421
:106AFD0068F583E493FF64636019AB3FAA40A94135
:106B0D00900002120721FEEF6E600890099BE004D1
:106B1D00F080CF90099BE0FF75F005A42418F58255
:106B2D00E43468F583E493601CEF75F005A4241933
:106B3D00F9746835F07548FFF549894A7B017A0982
:106B4D00796212AA84AB3FAA40A9419000011207B5
:106B5D00216066E490099BF090099BE075F005A417
:106B6D00244AF582E43468F583E493FF6019AB3F62
:106B7D00AA40A941900001120721FEEF6E60089016
:106B8D00099BE004F080D190099BE0FF75F005A40E
:106B9D00244AF582E43468F583E493601CEF75F0C4
:106BAD0005A4244BF9746835F07548FFF549894AF9
:106BBD007B017A09796212AA847B017A09796212C2
:106BCD00000E90099CEFF0AB3FAA40A941120708B7
:106BDD0014601D14606424FE7003026C972404601D
:106BED0003026D2E7BFF7A67793912B12E026D2E5D
:106BFD00AB3FAA40A94190000412072190099C3097
:106C0D00E11CE0FFC3740A9FF548AB42AA43A944B7
:106C1D00120708F5497BFF7A677944026D2BE0FF77
:106C2D00C3740A9FF548AB42AA43A944120708F55D
:106C3D00497BFF7A67794A026D2BAB3FAA40A94188
:106C4D0090000412072190099C30E11FE0FFC374EE
:106C5D000A9FF548AB42AA43A94412081FF54A857D
:106C6D00F0497BFF7A677950026D2BE0FFC3740A00
:106C7D009FF548AB42AA43A94412081FF54A85F077
:106C8D00497BFF7A677955026D2BAB3FAA40A9412D
:106C9D0090000412072130E03390099CE0FFC3748B
:106CAD000A9FF548900010120721FF600280027FB5
:106CBD00038F49AB42AA43A9441209218F4D8E4C33
:106CCD008D4B8C4A7BFF7A67795A8052AB3FAA4035
:106CDD00A94190000412072190099C30E121E0FFA9
:106CED00C3740A9FF548AB42AA43A9441209218FE8
:106CFD004C8E4B8D4A8C497BFF7A677962801FE001
:106D0D00FFC3740A9FF548AB42AA43A94412092157
:106D1D008F4C8E4B8D4A8C497BFF7A677968125464
:0A6D2D00967B017A09796212B12EFB
:016D37002239
:0D29660090098EE0FBA3E0FAA3E0F97DFFED
:102973008D428B3F8A4089419000011207216438C0
:102983007003023177AB3FAA40A94112070824FE26
:102993007003022BD824FE7003022E31240360033C
:1029A30002317790000412072120E103022A92AB3F
:1029B3003FAA40A9419000191209F0C000C001C00C
:1029C30002C003AC42EC1203BBD003D002D001D04F
:1029D3000012019EC004C005C006C007900938E07C
:1029E300FC1203BBD003D002D001D0001200AD1201
:1029F30003EF900938EFF0AB3FAA40A941900015CF
:102A03001209419000111209F012034470030231BC
:102A130077AB3FAA40A941900011120941C004C0FD
:102A230005C006C007900938E0FC1203BBA804A93F
:102A330005AA06AB07D007D006D005D0041203447D
:102A43005014AB3FAA40A94190001112094112034F
:102A5300EF900938EFF0AB3FAA40A941900015125F
:102A63000941C004C005C006C007900938E0FC1244
:102A730003BBA804A905AA06AB07D007D006D00557
:102A8300D00412034460025003023177022BC3E5E2
:102A930042F4704CAB3FAA40A94190001112094186
:102AA300C004C005C006C007900938E0FCE4120367
:102AB300BBA804A905AA06AB07D007D006D005D04A
:102AC30004120344701AAB3FAA40A94190001512A7
:102AD30009419000111209F0120344600302317797
:102AE300AB3FAA40A9419000191209F0C000C001F0
:102AF300C002C003AC42EC1203BBD003D002D0012E
:102B0300D00012019EC004C005C006C0079009385A
:102B1300E0FCE41203BBD003D002D001D0001200CA
:102B2300AD1203EF900938EFF0AB3FAA40A94190F3
:102B330000151209419000111209F01203447003A9
:102B4300023177AB3FAA40A941900011120941C05D
:102B530004C005C006C007900938E0FCE41203BBBB
:102B6300A804A905AA06AB07D007D006D005D00450
:102B73001203445014AB3FAA40A94190001112091B
:102B8300411203EF900938EFF0AB3FAA40A94190FF
:102B93000015120941C004C005C006C007900938DA
:102BA300E0FCE41203BBA804A905AA06AB07D007FF
:102BB300D006D005D00412034460025003023177DB
:102BC300AB3FAA40A9419000151209411203EF90AF
:102BD3000938EFF022AB3FAA40A941900004120745
:102BE3002120E103022CD69000191209F0C000C085
:102BF30001C002C003AC42EC1203BBD003D002D02D
:102C030001D00012019EC004C005C006C007900990
:102C130038E0FCA3E0FDEC1203B6D003D002D001F0
:102C2300D0001200AD1203EF900938EEF0A3EFF0DD
:102C3300AB3FAA40A941900015120941900011121F
:102C430009F01203447003023177AB3FAA40A94154
:102C5300900011120941C004C005C006C0079009C5
:102C630038E0FCA3E0FDEC1203B6A804A905AA060C
:102C7300AB07D007D006D005D0041203445017ABDE
:102C83003FAA40A9419000111209411203EF900994
:102C930038EEF0A3EFF0AB3FAA40A9419000151224
:102CA3000941C004C005C006C007900938E0FCA371
:102CB300E0FDEC1203B6A804A905AA06AB07D007EA
:102CC300D006D005D00412034460025003023177CA
:102CD300022E19E542F4704FAB3FAA40A941900080
:102CE30011120941C004C005C006C007900938E0AD
:102CF300FCA3E0FDE41203B6A804A905AA06AB07EA
:102D0300D007D006D005D004120344701AAB3FAAF3
:102D130040A9419000151209419000111209F012C7
:102D230003446003023177AB3FAA40A941900019E5
:102D33001209F0C000C001C002C003AC42EC120390
:102D4300BBD003D002D001D00012019EC004C00545
:102D5300C006C007900938E0FCA3E0FDE41203B607
:102D6300D003D002D001D0001200AD1203EF9009BE
:102D730038EEF0A3EFF0AB3FAA40A9419000151243
:102D830009419000111209F01203447003023177D4
:102D9300AB3FAA40A941900011120941C004C005EC
:102DA300C006C007900938E0FCA3E0FDE41203B6B7
:102DB300A804A905AA06AB07D007D006D005D004FE
:102DC3001203445017AB3FAA40A9419000111209C6
:102DD300411203EF900938EEF0A3EFF0AB3FAA40A6
:102DE300A941900015120941C004C005C006C007DF
:102DF300900938E0FCA3E0FDE41203B6A804A9059A
:102E0300AA06AB07D007D006D005D004120344604E
:102E1300025003023177AB3FAA40A941900015123B
:102E230009411203EF900938EEF0A3EFF022AB3F14
:102E3300AA40A94190000412072120E003022EF3C7
:102E4300900938E0F8A3E0F9A3E0FAA3E0FBC0009F
:102E5300C001C002C003AB3FAA40A94190001912B0
:102E630009F0C000C001C002C003AC42EC1203BBB6
:102E7300D003D002D001D00012019ED003D002D0E3
:102E830001D0001200AD900938120A2CAB3FAA40C2
:102E9300A941900011120941900938E0F8A3E0F923
:102EA300A3E0FAA3E0FB1203445012AB3FAA40A9EC
:102EB30041900011120941900938120A2CAB3FAA24
:102EC30040A941900015120941900938E0F8A3E0A8
:102ED300F9A3E0FAA3E0FB120344600250030231BA
:102EE30077AB3FAA40A94190001512094102317105
:102EF300AB3FAA40A94190000412072120E103023D
:102F0300300E9000191209F0C000C001C002C003C6
:102F1300AC42EC1203BBD003D002D001D0001201AB
:102F23009EC004C005C006C007900938E0FCA3E0BA
:102F3300FDA3E0FEA3E0FFEC1203B1D003D002D067
:102F430001D0001200AD1203EF900938120A2CAB26
:102F53003FAA40A94190001512094190001112099E
:102F6300F01203447003023177AB3FAA40A94190AA
:102F73000011120941C004C005C006C007900938FA
:102F8300E0FCA3E0FDA3E0FEA3E0FFEC1203B1A885
:102F930004A905AA06AB07D007D006D005D00412B2
:102FA30003445015AB3FAA40A941900011120941B7
:102FB3001203EF900938120A2CAB3FAA40A94190A3
:102FC3000015120941C004C005C006C007900938A6
:102FD300E0FCA3E0FDA3E0FEA3E0FFEC1203B1A835
:102FE30004A905AA06AB07D007D006D005D0041262
:102FF300034460025003023177AB3FAA40A94190DA
:1030030000151209411203EF023171E542F47055C4
:10301300AB3FAA40A941900011120941C004C00569
:10302300C006C007900938E0FCA3E0FDA3E0FEA3BF
:10303300E0FFE41203B1A804A905AA06AB07D00771
:10304300D006D005D004120344701AAB3FAA40A99E
:10305300419000151209419000111209F012034426
:103063006003023177AB3FAA40A9419000191209CE
:10307300F0C000C001C002C003AC42EC1203BBD0DD
:1030830003D002D001D00012019EC004C005C006C7
:10309300C007900938E0FCA3E0FDA3E0FEA3E0FF36
:1030A300E41203B1D003D002D001D0001200AD125C
:1030B30003EF900938120A2CAB3FAA40A9419000B4
:1030C300151209419000111209F012034470030212
:1030D3003177AB3FAA40A941900011120941C004C6
:1030E300C005C006C007900938E0FCA3E0FDA3E0DB
:1030F300FEA3E0FFE41203B1A804A905AA06AB07E7
:10310300D007D006D005D0041203445015AB3FAA14
:1031130040A9419000111209411203EF900938129E
:103123000A2CAB3FAA40A941900015120941C004E3
:10313300C005C006C007900938E0FCA3E0FDA3E08A
:10314300FEA3E0FFE41203B1A804A905AA06AB0796
:10315300D007D006D005D00412034460174015AB46
:103163003FAA40A9419000151209411203EF9009AB
:0531730038120A2C22B5
:10AE9C008F3FE92405F9E43AFA78627C097D017E5A
:10AEAC00007F081206E2E490096AF0900968E0FF5E
:10AEBC006007900967F0E4A3F0853F487549017578
:10AECC004A09754B627BFF7A67796E1254967BFF49
:07AEDC007A67797602B12EBE
:100BE600126FF9EF6003D21F22301F40E4900945CF
:100BF600F090093D120A5100000000900941120AC6
:100C06005100000000C222C223C224C225E490097A
:100C160094F012B362E47B2C7A01F9F8C31208FD52
:100C260040030216BFC21FD21412872E20271EC2EF
:100C36001412872E900994EFF070030216AFD22794
:100C4600E0640260030216AFD2260216AF20260326
:100C560002101D90096E742DF0E4A3F090097E74C5
:100C66002DF0E4A3F0754201754309754495754569
:100C760002FB7D02FF128DF6900995E0C4F854F050
:100C8600C868FCA3E0C4540F48FDE41203B6E4FBB5
:100C9600FAF978411202A7900997120A2CE4FFFE8E
:100CA6007D207C41900997E0F8A3E0F9A3E0FAA340
:100CB600E0FB12019EE4FBFAF9783F1200AD120345
:100CC600EFEC1203B1E4FBFA792078411202A79007
:100CD6000946120A2C7542017543097544957545F6
:100CE600027B017D02E4FF128DF6900995E0C4F8BF
:100CF60054F0C868FCA3E0C4540F48FDE41203B6E0
:100D0600E4FBFA79A0784012019EE4FBFA79807838
:100D1600451202A7900997120A2CE4FFFE7DC87CB3
:100D260042900997E0F8A3E0F9A3E0FAA3E0FB12EA
:100D3600019EE4FBFAF9783F1200AD1203EFEC12C4
:100D460003B1E4FBFA79C878421202A790094A1265
:100D56000A2C7542017543097544957545027B0257
:100D66007D02E4FF128DF6900995E0C4F854F0C8B0
:100D760068FCA3E0C4540F48FDE41203B6E4FBFA92
:100D86007920784012019EE4FBFA798078451202B8
:100D9600A7900997120A2C900997E0FCA3E0FDA3FF
:100DA600E0FEA3E0FF7B007AC0792878451202A70F
:100DB600900997120A2C900997E0FCA3E0FDA3E0A6
:100DC600FEA3E0FF7B007AC0795A784612019E9016
:100DD6000997120A2CE4FFFE7DC87C42900997E031
:100DE600F8A3E0F9A3E0FAA3E0FB12019EE4FBFA04
:100DF600F9783F1200AD1203EFEC1203B1E4FBFAEF
:100E060079C878421202A790094E120A2C7542013F
:100E16007543097544957545027B037D02E4FF120F
:100E26008DF6900995E0C4F854F0C868FCA3E0C4B8
:100E3600540F48FDE41203B6E4FBFA79C878401271
:100E4600019EE4FBFA798078451202A79009971271
:100E56000A2CE4FFFE7DC87C42900997E0F8A3E0E7
:100E6600F9A3E0FAA3E0FB12019EE4FBFAF9783F4E
:100E76001200AD1203EFEC1203B1E4FBFA79C87865
:100E8600421202A7900952120A2C754201754309B3
:100E96007544957545027B047D02E4FF128DF6903C
:100EA6000995E0C4F854F0C868FEA3E0C4540F489E
:100EB600FF7C007D0B120782AC06AD07E41203B679
:100EC600E4FBFA7920784012019EE4FBFA798078F7
:100ED600451202A7900997120A2CE4FFFE7DC87CF2
:100EE60042900997E0F8A3E0F9A3E0FAA3E0FB1229
:100EF600019EE4FBFAF9783F1200AD1203EFEC1203
:100F060003B1E4FBFA79C878421202A79009561297
:100F16000A2C7542017543097544957545027B0592
:100F26007D02E4FF128DF6900995E0C4F854F0C8EE
:100F360068FEA3E0C4540F48FF7C007D0B120782B5
:100F4600AC06AD07E41203B6E4FBFA79207840124A
:100F5600019EE4FBFA798078451202A79009971260
:100F66000A2CE4FFFE7DC87C42900997E0F8A3E0D6
:100F7600F9A3E0FAA3E0FB12019EE4FBFAF9783F3D
:100F86001200AD1203EFEC1203B1E4FBFA79C87854
:100F9600421202A790095A120A2C7542017543099A
:100FA6007544957545027B067D02E4FF128DF69029
:100FB6000995E0C4F854F0C868FCA3E0C4540F488F
:100FC600FDE41203B6E4FBFA7920784012019EE4B0
:100FD600FBFA798078451202A7900997120A2CE449
:100FE600FFFE7DC87C42900997E0F8A3E0F9A3E0F4
:100FF600FAA3E0FB12019EE4FBFAF9783F1200AD7A
:101006001203EFEC1203B1E4FBFA79C8784212023C
:10101600A790095E120A2C90098E30261374FFF0F1
:10102600A37468F0A374C7F0900992740CF080134F
:10103600E515F0A3E516F0A3E517F07882E614901F
:101046000992F0900992E0FFC394035005E4A3F0DF
:10105600801B900945E0FE7002800EEE900945B5B2
:101066000705E024FE8002E014900993F07882E6FA
:101076007014202611FDFF12B29A7BFF7A67797FE2
:101086001254960211D5E4900991F0900991E0FD71
:10109600C3940340030211D5E4FF12B29A9009915A
:1010A600E0FF900993E02FFFE433FE900945E07CD2
:1010B60000B50708ECB506047F1580027F2012B341
:1010C60026900991E0FD7F0112B29A900991E0FF06
:1010D600900993E02FFFE433FE900992E0FDD3EFF1
:1010E6009D7480F86E98400C7BFF7A677994125451
:1010F600960211CC900991E0FE900993E0FD2EFF37
:10110600C007EEFFED2FFFE433FEEF7805C333CEC5
:1011160033CED8F9FF90098EE0FBA3E0FAA3E02FC7
:10112600F9EA3EFAD00712AE9C900991E0FD7F0ADB
:1011360012B29A302040900991E0FF900993E02F77
:10114600FFE433FE900945E07C00B50729ECB506BF
:1011560025EF7805C333CE33CED8F9FF90098EE05C
:10116600FBA3E0FAA3E02FF9EA3EFA7542017543C4
:1011760009754438804D900991E0FF900993E02F5E
:10118600FFE433FEEF7805C333CE33CED8F9FF90B4
:10119600098EE0FBA3E0FAA3E02FF9EA3EFAC003CA
:1011A600C002C00190098EA3E0FAA3E02FF9EA3E3F
:1011B600FA90000D120AAC8B428A438944D001D0C2
:1011C60002D003126A67900991E004F00210919030
:1011D6000945E075F020A430260F24C7F974683558
:1011E600F0FA90098E74FF800D2517F9E51635F093
:1011F600FA90098EE515F0A3EAF0A3E9F030215A3A
:101206007D03E4FF12B29A7BFF7A6779A812B12EAA
:1012160090093CE075F003A4240DFF900993E0FECD
:10122600900945E0C39EFD12B29A20080A302207B3
:10123600C221E4FF12B39B2009030216AF30230339
:101246000216AF90093CE004F0E064036003021666
:10125600AFC221FF12B39B0216AF20200302142453
:101266007D03E4FF12B29A7BFF7A6779BD12B12E35
:10127600900993E0FF900945E0C39FFD7F1312B2EA
:101286009A20080A302207C220E4FF12B39B3009D5
:1012960053202350C220E4FF12B39B90098EE0FB3B
:1012A600A3E0FAA3E0F9120708FF7E0090098EA3D7
:1012B600A3E090000D120AACA801AC02AD037B01BD
:1012C6007A0979381206E2302612900945E0FF6065
:1012D60003B40110D228788076F18008900945E0A1
:1012E600FF12B2F8300A0F20240C12296612B362DC
:1012F60090093D120A2C300A2D12B362A804A905E2
:10130600AA06AB0790093DE0FCA3E0FDA3E0FEA31F
:10131600E02446FFE43EFEE43DFDE43CFCD3120837
:10132600FD4003122966300A3B12B362A804A905E0
:10133600AA06AB0790093DE0FCA3E0FDA3E0FEA3EF
:10134600E024F4FFEE3401FEE43DFDE43CFCD31260
:1013560008FD401090098EE0FBA3E0FAA3E0F97DBA
:10136600F7122973200A0A90093D120A510000005B
:1013760000300B1C20251990098EE0FBA3E0FAA390
:10138600E0F97D0112297312B362900941120A2C09
:10139600300B3A12B362A804A905AA06AB07900956
:1013A60041E0FCA3E0FDA3E0FEA3E02446FFE43E0B
:1013B600FEE43DFDE43CFCD31208FD401090098E8E
:1013C600E0FBA3E0FAA3E0F97D01122973300B3BA1
:1013D60012B362A804A905AA06AB07900941E0FC6E
:1013E600A3E0FDA3E0FEA3E024F4FFEE3401FEE457
:1013F6003DFDE43CFCD31208FD401090098EE0FB55
:10140600A3E0FAA3E0F97D09122973300B03021653
:10141600AF900941120A51000000000216AF7D0389
:10142600E4FF12B29A7882E6D3940050033026374E
:1014360090098EE0FBA3E0FAA3E0F99000191209E7
:1014460041E4FBFAF9F8120344401490098EE0FBDC
:10145600A3E0FAA3E0F990000412072130E2087B2A
:10146600FF7A6779D280067BFF7A6779DF12B12E21
:101476007F1212B3267BFF7A6779EC12B12E7F13A7
:1014860012B3267BFF7A6779F212B12E20080C3050
:101496002209C227C226D21412872E20090302155A
:1014A6008D30230302158D7882E6D3940040619037
:1014B600098EE0FBA3E0FAA3E0F9120708FFD39434
:1014C60004504DEF94004048900019120941E4FB86
:1014D600FAF9F81203445038D22090098EE0FBA3A3
:1014E600E0FAA3E0F9120708FF7E0090000D120A49
:1014F600AC78387C097D011206E2900993E0FF90F2
:101506000945E0C39FFD7F1312B29A7F0112B39B78
:1015160030262A900945E0FF64026004EFB4031DFB
:10152600D221E490093CF0900993E0FF900945E050
:10153600C39FFD7F0D12B29A7F0112B39B302637EF
:10154600900945E0640B702FD228788076F112B3AB
:10155600BAE4FDFF12B29A7BFF7A6779F412B12ED4
:101566007D01E4FF12B29A7BFF7A68790712B12EE9
:101576007FB87E0B12B10330260D900945E0B40CFE
:1015860006E4F58475EF10300A2A202427900945D1
:10159600E070122026077882E614F0800E90094546
:1015A600740CF08006900945E014F012B3629009BD
:1015B6003D120A2C300A4812B362A804A905AA06ED
:1015C600AB0790093DE0FCA3E0FDA3E0FEA3E02409
:1015D60046FFE43EFEE43DFDE43CFCD31208FD403C
:1015E6001E900945E070122026077882E614F080E6
:1015F6000E900945740CF08006900945E014F02021
:101606000A0A90093D120A5100000000302608908F
:101616000991740DF080077882E6900991F0300BFD
:1016260025202522900945E02401FFE433FE900998
:1016360091E0FD7C00120794900945EDF012B3622B
:10164600900941120A2C300B4312B362A804A90573
:10165600AA06AB07900941E0FCA3E0FDA3E0FEA3C8
:10166600E02446FFE43EFEE43DFDE43CFCD31208E4
:10167600FD4019900945E02401FFE433FE900991ED
:10168600E0FD7C00120794900945EDF0200B0A90CE
:101696000941120A5100000000300A0D300B0A20E1
:1016A6002607E4900945F0D226A2089222A20992C2
:0916B60023A20A9224A20B922542
:0116BF002208
:048DF6008D408B41E0
:108DFA007B08E4FD12B320E49009A3F0E54054088F
:108E0A00D394004003D38001C392B3000000000052
:108E1A00000000000000000000000000000000D276
:108E2A00B000000000000000000000000000000088
:108E3A000000000000C2B0E54025E0F5409009A31B
:108E4A00E004F0E0B404B5E49009A3F0E541540865
:108E5A00D394004003D38001C392B3000000000002
:108E6A00000000000000000000000000000000D226
:108E7A00B000000000000000000000000000000038
:108E8A000000000000C2B0E54125E0F5419009A3C9
:108E9A00E004F0E0B404B5E49009A3F0E54575F008
:108EAA0008A4FF9009A3E0FDC39FE5F06480F8746D
:108EBA008098505CED9400400FE05407700A042536
:108ECA0044F544E43543F543C2B000000000000015
:108EDA000000000000000000000000000000AB429B
:108EEA00AA43A94412070825E0FFA2B4E4334F12AB
:108EFA00074ED2B000000000000000000000000091
:108F0A0000000000000000009009A3E004F0808C3B
:108F1A00D2B20000000000000000000000000000C3
:068F2A0000000000000041
:018F3000221E
:049896007D0AAF4553
:04989A008D468B4725
:10989E00D2B2000000000000000000000000000036
:1098AE00000000000000C2B2000000000000000036
:1098BE000000000000000000000000007B08E4FD36
:1098CE0012B320E49009A3F0E5465408D394004067
:1098DE0003D38001C392B30000000000000000001B
:1098EE000000000000000000000000D2B0000000E8
:1098FE00000000000000000000000000000000005A
:10990E0000C2B0E54625E0F5469009A3E004F0E07C
:10991E00B404B5E49009A3F0E5475408D39400408D
:10992E0003D38001C392B3000000000000000000CA
:10993E000000000000000000000000D2B000000097
:10994E000000000000000000000000000000000009
:10995E0000C2B0E54725E0F5479009A3E004F0E02A
:03996E00B404B589
:0199710022D3
:10AD2300E4900992F0EF5480D394004003D3800160
:10AD3300C392B30000000000000000000000000008
:10AD430000000000000000D2B0000000000000007E
:10AD530000000000000000000000000000C2B0EF8F
:0DAD630025E0FF900992E004F0E0B408B88C
:01AD700022C0
:029B0F008F4580
:109B1100E4FB7D0712989AE4FB129896E4FF12ADDC
:109B210023E4FF12AD237B02129896E4FF12AD23CA
:109B3100E4FF12AD23E490098FF090098FE0FBC39D
:109B4100940750697D0CAF4512989A90098FE0FFF8
:109B5100700AA37403F0A37420F08017EF900990AA
:109B6100B402097401F0A374D9F08007740FF0A353
:109B710074FFF0900990E0C4F854F0C8A3E0C45415
:109B81000F48FF12AD23900991E0540FC4F8540F10
:109B9100C868FF12AD23E4FF12AD23E4FF12AD2329
:109BA1007F3A12AD2390098FE004F0808DE4FB7DB4
:109BB1000DAF4512989A7FFF12AD237FFF12AD239F
:0F9BC100E4FF12AD23E4FF12AD237F1402AD23A6
:10B20700E4FB7D0912989AD2B2000000000000000A
:0EB21700000000000000000000000000002207
:04B158008F1E8D1F9A
:10B15C007B017A0979B912A0EBE51F9009B9600659
:10B16C00E04401F08004E054FEF09009B9E0FDAF3A
:04B17C001E02A560AA
:10B2E0007B017A0979BAE4FF12A0EB9009BAE03049
:07B2F000E7037F00227F014C
:01B2F7002234
:10B2AE007B017A0979BBE4FF12A0EB9009BBE03079
:08B2BE00E704540FFF227F009A
:01B2C6002265
:10B25E007B017A0979BC12A0EB9009BCE0FFF46087
:0AB26E0007EF60047F0180027F00FB
:01B2780022B3
:03B3F10020200019
:0AAF1F00AB3FAA40A941120721FF31
:02AF29008F4750
:10AF2B00E478ACF6E5471392927F0A7E0012A90DE6
:10AF3B00D2937F0A7E0012A90DC293E547C313F586
:0AAF4B004778AC06E6C3940840DA2C
:01AF550022D9
:02A660008F77F2
:10A66200C293E4F58475D2FF75D30F7F0AFE12A957
:10A672000D75840F43A504AF7712AF2975840F536C
:10A68200A5FBD2927F0A7E0012A90DE478B0F618DB
:10A69200F678B1760130920778B0E679B147F6D212
:10A6A200937F0A7E0012A90DC2937F0A7E0012A92F
:10A6B2000D78B1E625E0F678AF06E6C3940840D5FA
:10A6C200E4F584F5D2F5D37F0AFE12A90D78B0E63F
:01A6D200FF88
:01A6D3002264
:069972008B3F8A40894191
:10997800C293E4F58475D2FF75D30F7F0AFE12A94E
:109988000D75840F43A5047FBF12AF2975840F534B
:10999800A5FBD2927F0A7E0012A90DE478A9F6E40D
:1099A80078AAF678A8F678AB760130920778AAE616
:1099B80079AB47F6D2937F0A7E0012A90DC2937F36
:1099C8000A7E0012A90D78ABE625E0F678A806E62F
:1099D800C3940840D578A9E6FFC39403501908E654
:1099E800FEEFFDC374059DFDE49400AB3FAA40A9BA
:1099F800418D82F583801E78A9E6FFC3940550182F
:109A080008E6FEEF7C0024FDF582EC34FFF583AB1D
:109A18003FAA40A941EE801178A9E6B4060E08E6EF
:109A2800AB3FAA40A94190000212076078A906E658
:109A3800C3940750030299A7E4F584F5D2F5D37FC0
:059A48000AFE02A90D59
:10AFC3008F458D46C293E4F58475D2FF75D30F7F09
:10AFD3000AFE12A90D75840F43A504AF4512AF29CC
:10AFE300AF4612AF29E4F584F5D2F5D37F0AFE020A
:02AFF300A90DA6
:10A5EA008B3F8A408941C293E4F58475D2FF75D3C3
:10A5FA000F7F0AFE12A90D75840F43A5047FBE12B0
:10A60A00AF2990000512AF1F90000412AF1FAB3F95
:10A61A00AA40A94190000312AF25AB3FAA40A94125
:10A62A00120708FF12AF29AB3FAA40A941900001C7
:10A63A0012AF257F0112AF29AB3FAA40A941900072
:10A64A000212AF25E4FF12AF29E4F584F5D2F5D35F
:06A65A007F0AFE02A90DBB
:10AEE3008D78EF14601614601914601C14601F141D
:10AEF300602224057025AD787F86801CAD787F881D
:10AF03008016AD787F8C8010AD787F84800AAD7811
:0CAF13007F828004AD787F8012AFC322E3
:1094D0008B188A19891A120708FFF47049AB1BAA66
:1094E0001CA91D900007743F120760900006743F8E
:1094F000120760900004743F120760900003743FED
:10950000120760900001743F120760743F12074E0B
:10951000AB1BAA1CA91D900005742D1207609000BA
:1095200002742D0295CDEFC4540F2430AB1BAA1C3E
:10953000A91D12074EAB18AA19A91A120708540F31
:109540002430AB1BAA1CA91D9000011207609000DB
:1095500002742D120760AB18AA19A91A9000011203
:109560000721C4540F2430AB1BAA1CA91D90000373
:10957000120760AB18AA19A91A900001120721540A
:109580000F2430AB1BAA1CA91D9000041207609089
:109590000005742D120760AB18AA19A91A900002D1
:1095A000120721C4540F2430AB1BAA1CA91D900024
:1095B00006120760AB18AA19A91A90000212072117
:1095C000540F2430AB1BAA1CA91D90000712076082
:0895D000900008E4120760227C
:1092AB008B688A69896A120708F47049AB6BAA6CE0
:1092BB00A96D900007743F120760900006743F126F
:1092CB000760900004743F120760900003743F1214
:1092DB000760900001743F120760743F12074EAB9A
:1092EB006BAA6CA96D900005743A1207609000028E
:1092FB00743A0293B5AB68AA69A96A900003120786
:10930B0021C4540F2430AB6BAA6CA96D12074EAB62
:10931B0068AA69A96A900003120721540F2430AB85
:10932B006BAA6CA96D900001120760900002743A51
:10933B00120760AB68AA69A96A900004120721C4DE
:10934B00540F2430AB6BAA6CA96D9000031207600D
:10935B00AB68AA69A96A900004120721540F243044
:10936B00AB6BAA6CA96D900004120760900005749A
:10937B003A120760AB68AA69A96A90000512072127
:10938B00C4540F2430AB6BAA6CA96D900006120766
:10939B0060AB68AA69A96A900005120721540F24D3
:1093AB0030AB6BAA6CA96D90000712076090000898
:0593BB00E4120760222E
:10ACD3007B017A0979A61299729009A6E0F4603F84
:10ACE300751B01751C09751DAC7B017A0979A612C8
:10ACF30094D07B017A0979AC12B12E7BFF7AB379B8
:10AD0300F112B12E756B01756C09756DAC7B017A0F
:0FAD13000979A61292AB7B017A0979AC12B12EA5
:01AD2200220E
:10B33C00E4FF12A660787EEFF6F460047F018002D1
:02B34C007F0080
:01B34E0022DC
:07000300E4FD7F8E02AFC394
:103178004C45442D4465627567004C45442D507597
:103188006C7365720044696E203556004F7074493F
:103198006E0043504C4400446F75742035562F32EE
:1031A80034560052656C616973004F70744F7574C2
:1031B8000055696E20302D322E35560055696E2027
:1031C8002B2D3130560049696E20302D322E356D49
:1031D800410049696E20302D32356D410055696EC8
:1031E80020302D322E3556204673740055696E20D6
:1031F8002B2D31305620466173740049696E20309A
:103208002D322E356D41204673740049696E203089
:103218002D32356D41204673740055696E202B2D73
:1032280031305620446966660055696E202B2D3171
:10323800305620466C740043696E20302D31306E54
:10324800460043696E20302D3175460050543130A8
:10325800302D38005054313030302D38004144354D
:1032680039300050543130302D3200505431303024
:10327800302D32004345524E4F582D3200554F7570
:103288007420302D322E355600554F7574202B2D55
:1032980031305600494F757420302D322E356D412E
:1032A80000494F757420302D32356D41004C6971DD
:1032B8002E4865206C6576656C00554F7574203214
:1032C80030305600245265763A203431363920247D
:1032D80000013400000050254F7574000000010003
:1032E800010000000000437F00003F800000000054
:1032F800000418000001502555696E2300000100E4
:1033080008040000000000000000000000000000A9
:10331800000418000001502555696E2300000100C3
:10332800040400000000000000000000000000008D
:10333800000418000001502555696E2300000100A3
:10334800020400000000000000000000000000006F
:10335800000418000001502555696E230000010083
:103368000804000000000000000000000000000049
:10337800000134000008502552616E6765000100A5
:103388000000000000000000000000000000000035
:103398000004180000015025556F757423000100C2
:1033A800080200000000402000003DCCCCCD000009
:1033B8000004180000015025556F757423000100A2
:1033C8000802C1200000412000003F00000000006A
:1033D800000406FD0001502549696E230000010024
:1033E80008040000000000000000000000000000C9
:1033F80000041DF70001502543696E2300000100F9
:1034080004040000000000000000000000000000AC
:1034180000040800000150255423000000000100AA
:10342800080200000000000000000000000000008A
:10343800000406FD00095025457863697400010001
:103448000001000000000000000000000000000073
:10345800000408000001502554230000000001006A
:10346800080200000000000000000000000000004A
:10347800000408000001502554230000000001004A
:103488000202000000000000000000000000000030
:10349800000407000001502554230000000001002B
:1034A8000202000000000000000000000000000010
:1034B800000406FD00015025496F757423000100C2
:1034C80008020000000041A000003DCCCCCD000067
:1034D800000406FD00095025457863697400010061
:1034E80000010000000042C800003F80000000000A
:1034F80000045A00000950254C4F66730000010073
:1035080000020000000000000000000000000000B1
:1035180000045D00000950254C4761696E000100F8
:103528000002000000000000000000000000000091
:103538000002030000085025546F66660000010071
:103548000000000000000000000000000000000073
:103558000002030000085025546F6E0000000100AF
:103568000000000000000000000000000000000053
:1035780000045A00000150254C696E00000001004B
:103588000001000000000000000000000000000032
:10359800000132000000502544696E23000001003C
:1035A800080100000000000000000000000000000A
:1035B800000132000000502544696E23000001001C
:1035C80004010000000000000000000000000000EE
:1035D8000001320000005025446F7574230001007B
:1035E8000801000000003F8000003F80000000004C
:1035F800000132000000502552656C2300000100D4
:103608000401000000003F8000003F80000000002F
:1036180000013200000050254F757423000001009E
:103628000401000000003F8000003F80000000000F
:103638000004180000015025554423000000010033
:10364800080300000000434800003F80000000001D
:103658000004180000015025552300000000010057
:103668000803000000000000000000000000000047
:10367800000406FA0001502549230000000001005B
:103688000803000000000000000000000000000027
:103698000001FF3178FF32D901FFAA2C02FF3182E5
:1036A8000000000100000020FF318DFF359901FF67
:1036B80093C021FF3194FF35B901FF93C022FF3138
:1036C8009AFF359901FF93C040FF319FFF35D9011B
:1036D800FF844B41FF31ABFF35F901FF844B42FFBB
:1036E80031B2FF361901FF844B60FF31B9FF32F95F
:1036F80001FF5CA261FF31C4FF32F901FF5CA262E5
:10370800FF31CEFF33D901FF5CA263FF31DAFF330B
:10371800D901FF5CA264FF31E5FF32F901FF607D4A
:1037280065FF31F4FF32F901FF607D66FF3203FF68
:1037380033D901FF607D67FF3213FF33D901FF6082
:103748007D68FF3222FF331901FF5CA269FF323125
:10375800FF333901FF755870FF323FFF33F901FF1E
:1037680072AC71FF324AFF33F901FF72AC72FF325B
:1037780054FF341902FF4F8173FF325CFF34190282
:10378800FF4F8174FF3265FF345901FF6D3875FFB3
:10379800326BFF347901FF4A6976FF3273FF34795F
:1037A80001FF4A6977FF327CFF349901FF4A69803B
:1037B800FF3285FF339901FF7C2E81FF3291FF3361
:1037C800B901FF450882FF329CFF34B901FF7C2E06
:1037D80083FF32A9FF34B901FF7C2E84FF32B5FF85
:1037E80034D906FF16C085FF32C2FF363903FF3EC3
:1037F800F000000000000000000000003CA3D70A11
:103808003D23D70A3DA3D70A3E23D70A3EA3D70AAA
:103818003F23D70A3FA3D70A4023D70A0504030248
:0C3828000100060706020703000405016A
:1082CE00E5792412F8E6FFE5792413F8E6FD7550FA
:0382DE00017B061B
:1082E100D2B1C2B0C2B2E49009A5F09009A5E0FEF6
:1082F100C39404504CEFC8EEC8088002C333D8FCC5
:108301005408D394004003D38001C392B30000000A
:10831100000000000000000000000000000000005C
:1083210000D2B000000000000000000000000000CA
:1083310000000000000000C2B09009A5E004F08038
:10834100AAE49009A5F09009A5E0FFC39403504C5D
:10835100EDC8EFC8088002C333D8FC5404D394009D
:108361004003D38001C392B300000000000000006D
:10837100000000000000000000000000D2B000007A
:1083810000000000000000000000000000000000EC
:108391000000C2B09009A5E004F080AAE49009A50C
:1083A100F09009A5E0FFC39404504CEBC8EFC80856
:1083B1008002C333D8FC5408D394004003D3800116
:1083C100C392B300000000000000000000000000A4
:1083D10000000000000000D2B0000000000000001A
:1083E10000000000000000000000000000C2B0908A
:1083F10009A5E004F080AAD2B2000000000000004C
:1084010000000000000000000000000000D2B000E9
:10841100000000000000000000000000000000005B
:10842100000000C2B0C2B2C2B3E55024FF92B0D284
:10843100B2C2B10000000000000000000000000016
:0984410000000000000000C2B2BE
:01844A00220F
:10B31000E5792409F8E6FFE579240AF8E6FD7B06DD
:06B32000E4F5500282E199
:05A33000F8E6FD7BFFD3
:03A33500CCEBCCA2
:10A338007B0312B320E490098EF0EC5480D3940090
:10A348004003D38001C392B3000000000000000066
:10A35800000000000000000000000000D2B0000073
:10A3680000000000000000000000000000000000E5
:10A378000000C2B0EC25E0FC90098EE004F0E0B4E7
:10A3880008B8C2B3D2B2000000000000000000000C
:10A3980000000000000000000000D2B00000000033
:10A3A80000000000000000000000000000000000A5
:04A3B800C2B0C2B2BB
:01A3BC00227E
:109D3500E5792405F8EFF6E5792412F8E6FFE579EB
:0C9D45002413F8E6FDE5792405F8E6FBA0
:039D5100CCEBCC8C
:109D54007B0212B320E490098EF0EC5480D394007B
:109D64004003D38001C392B3000000000000000050
:109D7400000000000000000000000000D2B000005D
:109D840000000000000000000000000000000000CF
:109D94000000C2B0EC25E0FC90098EE004F0E0B4D1
:109DA40008B8C2B3D2B200000000000000000000F6
:109DB40000000000000000000000D2B0000000001D
:109DC400000000000000000000000000000000008F
:049DD400C2B0C2B2A5
:019DD8002268
:0C9E7C00F8E6FD7B00E5792408F97A0087
:069E88008B448A45894667
:109E8E00E4FB12B320D2B20000000000000000007C
:109E9E000000000000000000000000D2B000000032
:109EAE0000000000000000000000000000000000A4
:109EBE0000C2B0C2B2E490098EF0000000000000B3
:109ECE000000000000000000000000000000D2B002
:109EDE000000000000000000000000000000000074
:109EEE0000000000C2B090098FE025E0FFA2B4E4AC
:109EFE00334FF090098EE004F0E0B408BD90098F66
:0A9F0E00E0AB44AA45A94602074E45
:06A2A0008B448A4589464B
:10A2A6007B0112B320D2B2000000000000000000C3
:10A2B6000000000000000000000000D2B000000016
:10A2C6000000000000000000000000000000000088
:10A2D60000C2B0C2B2E490098EF000000000000097
:10A2E6000000000000000000000000000000D2B0E6
:10A2F6000000000000000000000000000000000058
:10A3060000000000C2B090098FE025E0FFA2B4E48F
:10A31600334FF090098EE004F0E0B408BD90098F49
:0AA32600E0AB44AA45A94602074E29
:03A56000CCEDCC73
:10A563007B05E4FD12B320E49009BDF0EC5480D3E5
:10A5730094004003D38001C392B3000000000000A5
:10A583000000000000000000000000000000D2B046
:10A5930000000000000000000000000000000000B8
:10A5A30000000000C2B0EC25E0FC9009BDE004F01F
:10A5B300E0B408B8C2B3D2B200000000000000004B
:10A5C300000000000000000000000000D2B0000006
:10A5D3000000000000000000000000000000000078
:06A5E3000000C2B0C2B28C
:01A5E900224F
:06A0EB008B3F8A40894111
:10A0F1007B04E4FD12B320D2B20000000000000096
:10A1010000000000000000000000000000D2B000CC
:10A11100000000000000000000000000000000003E
:10A12100000000C2B0C2B2E49009A3F00000000038
:10A13100000000000000000000000000000000001E
:10A14100D2B000000000000000000000000000008C
:10A15100000000000000C2B09009A4E025E0FFA2C9
:10A16100B4E4334FF09009A3E004F0E0B408BD90EB
:0CA1710009A4E0AB3FAA40A94102074E40
:10B2C7007B017A09798C128CB590098CE0D39400B4
:08B2D70040047F0180027F00AA
:01B2DF00224C
:068CB5008B448A4589464C
:108CBB007B0712B320D2B3000000000000000000BD
:108CCB000000000000000000000000D2B000000017
:108CDB000000000000000000000000000000000089
:108CEB0000C2B0D2B3000000000000000000000082
:108CFB00000000000000000000D2B00000000000E7
:108D0B00000000000000000000000000000000C296
:108D1B00B0C2B30000000000000000000000000023
:108D2B0000000000000000D2B000000000000000B6
:108D3B0000000000000000000000000000C2B0E4D2
:108D4B0090098DF0C2B3000000000000000000008D
:108D5B0000000000000000000000D2B00000000086
:108D6B0000000000000000000000000000000000F8
:108D7B00C2B090098DE004F0E0B406C830B409AB82
:108D8B0044AA45A946E4805FE490098DF0000000F9
:108D9B0000000000000000000000000000000000C8
:108DAB0000D2B00000000000000000000000000036
:108DBB0000000000000000C2B090098FE025E0FF2A
:108DCB0090098EE033FEA2B4E433FDEF4DFFEEF0DD
:108DDB00A3EFF090098DE004F0E0B410B090098E91
:0A8DEB00E0AB44AA45A94612074E6A
:018DF500225B
:10AF5600900989EFF0A3EDF0A3EBF012B2C7EF7002
:10AF660002FF22900989E0FFA3E0FD7B017A0979BF
:10AF760088128CB590098BE0FF900988E06F700409
:06AF86007F0180027F0044
:01AF8C0022A2
:0377FA00CCEBCC09
:1077FD007B0712B320D2B300000000000000000090
:10780D000000000000000000000000D2B0000000E9
:10781D00000000000000000000000000000000005B
:10782D0000C2B0C2B3000000000000000000000064
:10783D00000000000000000000D2B00000000000B9
:10784D00000000000000000000000000000000C269
:10785D00B0C2B300000000000000000000000000F6
:10786D0000000000000000D2B00000000000000089
:10787D0000000000000000000000000000C2B0E4A5
:10788D009009B6F0D2B30000000000000000000027
:10789D0000000000000000000000D2B00000000059
:1078AD0000000000000000000000000000000000CB
:1078BD00C2B09009B6E004F0E0B406C8D2B2000040
:1078CD0000000000000000000000000000000000AB
:1078DD000000C2B2D2B300000000000000000000A2
:1078ED0000000000000000000000D2B00000000009
:1078FD00000000000000000000000000000000007B
:10790D00C2B0C2B300000000000000000000000083
:10791D000000000000000000D2B0000000000000D8
:10792D000000000000000000000000000000C2B0D8
:10793D00D2B30000000000000000000000000000B5
:10794D00000000000000D2B00000000000000000A8
:10795D00000000000000000000000000C2B0E49034
:10796D0009B6F0C2B30000000000000000000000E6
:10797D00000000000000000000D2B0000000000078
:10798D00000000000000000000000000000000C228
:10799D00B09009B6E004F0E0B406C8E49009B6F082
:1079AD00EC5480D394004003D38001C392B3000004
:1079BD0000000000000000000000000000000000BA
:1079CD000000D2B000000000000000000000000028
:1079DD000000000000000000C2B0EC25E0FC9009A2
:1079ED00B6E004F0E0B410B8D2B200000000000020
:1079FD000000000000000000000000000000C2B206
:0A7A0D00E49009B7F0A3F020B427BD
:0D7A170075750175760300D576FCD575F602
:107A24009009B8E004F070069009B7E004F09009FA
:0A7A3400B7E0B427DBA3E0B410D6DE
:017A3E002225
:10844B001579A879EBF61579A879EDF61579A87950
:04845B00EFF61579AA
:10845F00A8790808E6640160030284EDE579240435
:10846F00F8E6FEE5792403F8E6FF75F008A42EF58B
:10847F0082E435F0F583E5822418F582E583340034
:10848F00F583E4F0F584E5EF20E119E5792404F8AC
:10849F00E6FDEF75F008A42D2418F9E43400FA7BFB
:1084AF000112A2A0E5792403F8E6FFE5792404F888
:1084BF00E6FD75F008EFA42DF582E435F0F583E5C0
:1084CF00822418F582E5833400F583E0FB129D5179
:1084DF00E5792403F8E6FFE579240412A330A8799F
:1084EF000808E6640260030285B6E5792406F8CB36
:1084FF00E6CB08E6FA08E6F9120708A879F6603E17
:10850F00E5792404F8E6FFE5792403F8E675F00829
:10851F00A42FF582E435F0F583E5822418F582E582
:10852F00833400F583E0FFE5792405F8E6FE740156
:10853F00C8EEC8088002C333D8FC4FF0803DE57900
:10854F002404F8E6FFE5792403F8E675F008A42F74
:10855F00F582E435F0F583E5822418F582E583345E
:10856F0000F583E0FFE5792405F8E6FE7401C8EE17
:10857F00C8088002C333D8FCF45FF0E5792403F810
:10858F00E6FFE5792404F8E6FD75F008EFA42DF574
:10859F0082E435F0F583E5822418F582E583340013
:0985AF00F583E0FB129D517F00F1
:0785B800E5792409F57922A1
:1093C0001579A879EBF61579A879EDF61579A879CC
:0493D000EFF6157926
:1093D400A8790808E6640360030294C7E5792406C3
:1093E400F8CBE6CB08E6FA08E6F9120708603EE592
:1093F400792404F8E6FFE5792403F8E675F008A477
:109404002FF582E435F0F583E5822418F582E583AF
:109414003400F583E0FFE5792405F8E6FE7401C81D
:10942400EEC8088002C333D8FC4FF0803DE57924B0
:1094340004F8E6FFE5792403F8E675F008A42FF5AF
:1094440082E435F0F583E5822418F582E58334005F
:10945400F583E0FFE5792405F8E6FE7401C8EEC85B
:10946400088002C333D8FCF45FF0E5792403F8E6FE
:10947400FFE5792404F8E6FD7B00A9797A00129EC1
:1094840088E5792405F974017E00C8E7C8088005D9
:10949400C333CE33CED8F9FFA879E6FDEF5DD3947C
:1094A400007480948040047F0180027F00E5792469
:1094B40006F8CBE6CB08E6FA08E6F9EF12074E7F8A
:0594C4000180027F00A1
:0794C900E5792409F5792281
:10AA2C001579A879EBF61579A879EDF61579A87949
:10AA3C00EFF6A87908E6B4010DA8790808E6FFE559
:10AA4C0079240312A330A87908E6B40222A8790865
:10AA5C0008E6FFE5792403F8E6FDE5792405F8CB53
:10AA6C00E6CB08E6FA08E6F9120708FB129D517FBF
:08AA7C0000E5792408F57922B8
:107C2E001579A879EBF61579A879EDF61579A87975
:087C3E00EFF6E57924F9F57970
:107C46002408F8E664026003027DEDE579240CF869
:107C5600CBE6CB08E6FA08E6F9120921A879120A5A
:107C660020E5792407F8E6B40209E4FBFA79C87836
:107C7600428022E5792407F8E6B48209E4FBFA7922
:107C86002078408010E5792407F8E6B4832DE4FBDC
:107C9600FA79C87841E8C0E0A8791209AFD0E0F8CF
:107CA6001202A77B007AFF797F784712019E1203A2
:107CB600EFE5792404F8EEF608EFF612B310E5794D
:107CC6002406F8E4F6E5792406F8E6FFC3940450A2
:107CD6003FEF94014003D38001C392B3000000003C
:107CE600000000000000000000000000000000008E
:107CF600D2B00000000000000000000000000000FC
:107D0600000000000000C2B0E5792406F80680B540
:107D1600E5792406F8E4F6E5792406F8E6C3940442
:107D26005051E579240BF8E6FF5408D3940040033C
:107D3600D38001C392B300000000000000000000E1
:107D460000000000000000000000D2B000000000AB
:107D5600000000000000000000000000000000001D
:107D6600C2B0E579240BF8EF25E0F6E5792406F8AC
:107D76000680A4E5792406F8E4F6E5792406F8E613
:107D8600C394105060E5792404F8E6FE08E6FFEE99
:107D96005480FCD3E49400EC94004003D38001C3E8
:107DA60092B3000000000000000000000000000088
:107DB600000000000000D2B000000000000000003B
:107DC600000000000000000000000000C2B0E579DD
:107DD6002404F8EF25E0FFEE33F608EFF6E5792404
:097DE60006F8068095D2B17F0079
:077DEF00E579240FF579226C
:104508001579A879EBF61579A879EDF61579A879D2
:08451800EFF6E57924F9F579CD
:10452000E5792408F8E664026003024A60E579242C
:104530000CF8CBE6CB08E6FA08E6F9120921A879CF
:10454000120A20E4FFFE7D207C41A8791209C712DF
:104550000344600B4009A879120A3841200000E4A6
:10456000FFFE7D207CC1A8791209C71203445009BF
:10457000A879120A38C1200000E4FFFE7D207C41AA
:10458000A8791209C71200ADE4FBFA79A0784112AC
:1045900002A77B007AFF797F784712019EE4FBFA3D
:1045A000F9783F1200AD1203EFE5792404F8EEF636
:1045B00008EFF612B310C2B30000000000000000C4
:1045C000000000000000000000000000D2B0000069
:1045D00000000000000000000000000000000000DB
:1045E0000000C2B0C2B300000000000000000000E4
:1045F00000000000000000000000D2B00000000039
:1046000000000000000000000000000000000000AA
:10461000C2B0E579240BF8E6FFC394045049E5796C
:104620002406F8E4F6E5792406F8E6C39416400378
:1046300002480A0000000000000000000000000026
:1046400000000000000000D2B000000000000000E8
:1046500000000000000000000000000000C2B0E503
:10466000792406F80680BEC2B300000000000000F6
:1046700000000000000000000000000000D2B000B8
:10468000000000000000000000000000000000002A
:10469000000000C2B0D2B300000000000000000023
:1046A0000000000000000000000000D2B000000088
:1046B00000000000000000000000000000000000FA
:1046C00000C2B0C2B3000000000000000000000003
:1046D000000000000000000000D2B0000000000058
:1046E000000000000000000000000000000000C208
:1046F000B0C2B30000000000000000000000000095
:1047000000000000000000D2B00000000000000027
:1047100000000000000000000000000000C2B0EF38
:104720005402D394004003D38001C392B30000002D
:104730000000000000000000000000000000000079
:1047400000D2B000000000000000000000000000E7
:1047500000000000000000C2B0E579240BF8E65428
:1047600001D394004003D38001C392B30000000042
:104770000000000000000000000000000000000039
:10478000D2B00000000000000000000000000000A7
:10479000000000000000C2B0E5792406F8E4F6E568
:1047A000792406F8E6C394105060E5792404F8E60D
:1047B000FE08E6FFEE5480FCD3E49400EC94004045
:1047C00003D38001C392B30000000000000000008A
:1047D0000000000000000000000000D2B000000057
:1047E00000000000000000000000000000000000C9
:1047F00000C2B0E5792404F8EF25E0FFEE33F608B7
:10480000EFF6E5792406F8068095C2B300000000B3
:104810000000000000000000000000000000000098
:10482000D2B0000000000000000000000000000006
:10483000000000000000C2B0C2B300000000000091
:104840000000000000000000000000000000D2B0E6
:104850000000000000000000000000000000000058
:1048600000000000C2B0E579240BF8E6FFD3940302
:104870004049E5792406F8E4F6E5792406F8E6C32C
:1048800094164003024A5E00000000000000000091
:104890000000000000000000000000D2B000000096
:1048A0000000000000000000000000000000000008
:1048B00000C2B0E5792406F80680BEC2B30000004D
:1048C00000000000000000000000000000000000E8
:1048D00000D2B00000000000000000000000000056
:1048E00000000000000000C2B0D2B30000000000D1
:1048F000000000000000000000000000000000D2E6
:10490000B0000000000000000000000000000000F7
:104910000000000000C2B0C2B300000000000000B0
:1049200000000000000000000000000000D2B00005
:104930000000000000000000000000000000000077
:10494000000000C2B0C2B300000000000000000080
:104950000000000000000000000000D2B0000000D5
:104960000000000000000000000000000000000047
:1049700000C2B0EF5402D394004003D38001C3922D
:10498000B300000000000000000000000000000074
:104990000000000000D2B000000000000000000095
:1049A0000000000000000000000000C2B0E5792413
:1049B0000BF8E65401D394004003D38001C392B3B3
:1049C00000000000000000000000000000000000E7
:1049D00000000000D2B00000000000000000000055
:1049E00000000000000000000000C2B0E5792406CD
:1049F000F8E4F6E5792406F8E6C394105060E5790A
:104A00002404F8E6FE08E6FFEE5480FCD3E49400AC
:104A1000EC94004003D38001C392B3000000000077
:104A2000000000000000000000000000000000D2B4
:104A3000B0000000000000000000000000000000C6
:104A40000000000000C2B0E5792404F8EF25E0FF83
:104A5000EE33F608EFF6E5792406F8068095D2B134
:024A60007F00D5
:074A6200E579240FF579222C
:0B89FF007D527F03128A0A7D037F0176
:108A0A001579A879EDF61579A879EFF6157915791A
:108A1A00C2B3C2B100000000000000000000000064
:108A2A000000000000000000A879E4F6A879E6C377
:108A3A0094045031C2B0C2B300000000000000002C
:108A4A00000000000000000000000000D2B000009A
:108A5A00000000000000000000000000000000000C
:108A6A0000000680C7A879E4F6A879087608A879EC
:108A7A00E6C39404504AC2B008E6FFA8790808562B
:108A8A0094004003D38001C392B3000000000000A9
:108A9A000000000000000000000000000000D2B04A
:108AAA0000000000000000000000000000000000BC
:108ABA0000000000A87908EFC313F6A8790680AE73
:108ACA00D2B2000000000000000000000000000018
:108ADA00000000000000C2B2A879E4F6A87908767E
:108AEA0080A879E6C39408504DC2B008E6FFE5793C
:108AFA002403F8E65FD394004003D38001C392B302
:108B0A00000000000000000000000000000000005B
:108B1A0000000000D2B000000000000000000000C9
:108B2A0000000000000000000000A87908EFC3134D
:108B3A00F6A8790680ABD2B1C2B3000000000000EB
:0E8B4A0000000000000000000000000000001D
:078B5800E5792404F5792200
:0A9F18001579A879EFF6157915798F
:109F2200C2B3C2B100000000000000000000000047
:109F32000000000000000000A879E4F6A879087685
:109F420080A879E6C39408504AC2B008E6FFA8790F
:109F520008085694004003D38001C392B300000066
:109F620000000000000000000000000000000000EF
:109F720000D2B0000000000000000000000000005D
:109F820000000000000000A87908EFC313F6A879CA
:109F92000680AED2B1C2B300000000000000000093
:0B9FA2000000000000000000000000B4
:079FAD000579057905792211
:0B7DF6007B00E5792409F97A007F0486
:107E0100157915791579A879C6EBC608C6EAC608A9
:0D7E1100C6E9C61579A879EFF6157915793F
:107E1E00C2B10000000000000000000000000000E1
:107E2E00000000000000A879E4F6A879E6FFC394EC
:107E3E0004503BC2B0EFB40103D38001C392B30030
:107E4E000000000000000000000000000000000024
:107E5E00000000D2B0000000000000000000000092
:107E6E00000000000000000000A8790680BCA87980
:107E7E00E4F6A879087608A879E6C39404504AC2B5
:107E8E00B008E6FFA87908085694004003D3800195
:107E9E00C392B300000000000000000000000000CC
:107EAE0000000000000000D2B00000000000000042
:107EBE0000000000000000000000000000A879088B
:107ECE00EFC313F6A8790680AED2B2000000000010
:107EDE00000000000000000000000000000000C2D2
:107EEE00B2A879E4F6E5792403F8CBE6CB08E6FAF6
:107EFE0008E6F9120A8200000000A879E6C3941879
:107F0E005070C2B000000000000000000000000031
:107F1E000000000000000000E5792403F8CBE6CB5A
:107F2E0008E6FA08E6F9120921780112090EC8ECE2
:107F3E00C8C9EDC9CAEECACBEFCBA2B4E4334BFF2E
:107F4E00EAFEE9FDE8FCE5792403F8CBE6CB08E68A
:107F5E00FA08E6F9120971D2B00000000000000024
:107F6E0000000000000000000000000000A87906DC
:107F7E008088D2B100000000000000000000000068
:087F8E000000000000000000EB
:077F9600E5792406F57922CC
:105CA2001579A879EBF61579A879EDF61579A87921
:085CB200EFF6E57924F5F57920
:105CBA00240CF8E664016003025D7DE579240DF8A1
:0C5CCA00E6FFE579240E1282D91289FF52
:105CD600E5792409F87664E5792409F8E6D3940091
:105CE6004023E579240AF87603E579240AF8E6D311
:105CF6009400400900E579240AF81680ECE5792439
:055D060009F81680D22F
:105D0B00E579240EF8E6FFE579240DF8E6FE75F04B
:105D1B0008A42FF582E435F0F583E5822478F5822B
:105D2B00E5833400F5837407F075F008EEA42FF5C6
:105D3B0082E435F0F583E5822478F582E58334003F
:105D4B00F583E04408FD7F02128A0AE579240EF8F8
:105D5B00E6FFE579240DF8E675F008A42FF582E44B
:105D6B0035F0F583E5822490F582E5833403F583E2
:105D7B00E4F0E579240CF8E6FF64027042E579243F
:105D8B000FF8E6B40839E5792410F8CBE6CB08E632
:105D9B00FA08E6F9120708FEE579240EF8E6FDE5A8
:105DAB0079240DF8E675F008A42DF582E435F0F5AD
:105DBB0083E5822478F582E5833400F583EEF0EFFA
:105DCB0064036003026074E579240FF8E6D394074B
:105DDB0040057F00026076E579240DF8E6FFE57952
:105DEB00240E129E7CE5792408F8E65401D3940026
:105DFB0040057F00026076E579240EF8E6FDE57933
:105E0B00240DF8E6FE75F008A42DF582E435F0F5C7
:105E1B0083E5822490F582E5833403F583E0FFE587
:105E2B0079240FF8E66F60057F00026076CFEECF26
:105E3B001282DC7B00E5792404127DFCE579240BCE
:105E4B00F8E66468702CE579240EF8E6FFE5792412
:105E5B000DF8E6FE75F008A42FF582E435F0F58316
:105E6B00E5822490F582E5833403F583E004540343
:105E7B00802AE579240EF8E6FFE579240DF8E6FE95
:105E8B0075F008A42FF582E435F0F583E5822490B4
:105E9B00F582E5833403F583E0045407FD75F008C0
:105EAB00EEA42FF582E435F0F583E5822490F5829C
:105EBB00E5833403F583EDF0E579240EF8E6FFE591
:105ECB0079240DF8E6FE75F008A42FF582E435F081
:105EDB00F583E5822490F582E5833403F583E0C4F2
:105EEB0054F04408FD75F008EEA42FF582E435F06C
:105EFB00F583E5822478F582E5833400F583E04D64
:105F0B00FD7F02128A0AE5792404F81209AFE41224
:105F1B0003B1E4FBFA7980784B1202A7E579240EE2
:105F2B00F8E6FBE579240DF8E675F008A42BF5826D
:105F3B00E435F0F583E5822478F582E5833400F5CA
:105F4B0083E025E025E02404F582E43438F5831260
:105F5B0009E012019EA879120A20E579240BF8E6D4
:105F6B00B460028014E579240BF8E6B46102804337
:105F7B00E579240BF8E6B46211A879E8C0E01209C0
:105F8B00AFE4FBFA7980783F8018E579240BF8E6CB
:105F9B00B46317A879E8C0E01209AFE4FBFA7920E3
:105FAB00784112019ED0E0F88034E579240BF8E6B5
:105FBB00B4682EE4FBFA79207840E8C0E0A87912A7
:105FCB0009AFD0E0F81202A7E4FBFA79A0784112EE
:105FDB00019EE4FBFA792078C11200ADA879120A70
:105FEB0020E579240BF8E6FF64616009EF646360D8
:105FFB0004EFB4682A7F007E507DC37C47A87912DA
:10600B0009C712019EE4FBFAF9783F1200AD1203A7
:10601B00EFEC1203B17B007A5079C3784780287F6D
:10602B00007E247D747C49A8791209C712019EE475
:10603B00FBFAF9783F1200AD1203EFEC1203B17BC0
:10604B00007A24797478491202A7A879120A20A839
:10605B00791209AFE5792410F8CBE6CB08E6FA08FC
:0B606B00E6F91209717F0480027F003B
:07607600E5792413F57922FE
:104F81001579A879EBF61579A879EDF61579A8794F
:084F9100EFF6E57924F1F57952
:104F99002410F8E66401600302502DE5792411F824
:0C4FA900E6FFE57924121282D91289FF7C
:104FB500E579240DF87664E579240DF8E6D39400B7
:104FC5004023E579240EF87603E579240EF8E6D337
:104FD5009400400900E579240EF81680ECE5792463
:054FE5000DF81680D25A
:104FEA007D0F7F02128A0AE5792412F8E6FFE57935
:104FFA002411F8E675F008A42FF582E435F0F5835C
:10500A00E5822400F582E5833400F583E4F0EF2598
:10501A00E025E02490F582E43400F583120A513F3A
:10502A00800000E5792410F8E6640260030250F07B
:10503A00E5792413F8E6640860030250F0E5792460
:10504A0014F8CBE6CB08E6FA08E6F9120921E57965
:10505A002412F8E6FB25E025E02490F582E43400EA
:10506A00F583120A2CEB25E025E02490F582E4343E
:10507A0000F583E0FCA3E0FDA3E0FEA3E0FF7B0ACA
:10508A007AD77923783C1203446002502AE57924BE
:10509A0012F8E625E025E02490F582E43400F58351
:1050AA00E0FCA3E0FDA3E0FEA3E0FFE4FBFA792025
:1050BA007841120344502FE5792412F8E625E025B9
:1050CA00E02490F582E43400F583120A513F80000F
:1050DA0000E5792414F8CBE6CB08E6FA08E6F912DB
:1050EA000A823F800000E5792410F8E66403600331
:1050FA0002542BE5792413F8E6D3940740057F0080
:10510A0002542DE5792411F8E6FFE5792412129E5E
:10511A007CE5792408F8E65401D3940040057F0021
:10512A0002542DE5792412F8E6FDE5792411F8E612
:10513A00FE75F008A42DF582E435F0F583E58224A6
:10514A0000F582E5833400F583E0FFE5792413F85E
:10515A00E66F60057F0002542DCFEECF1282DC127B
:10516A007DF6E5792412F8E6FFE5792411F8E6FEE2
:10517A0075F008A42FF582E435F0F583E582240062
:10518A00F582E5833400F583E0045407FD75F008E1
:10519A00EEA42FF582E435F0F583E5822400F5824A
:1051AA00E5833400F583EDF0E5792412F8E6FFE5AE
:1051BA00792411F8E675F008A42FF582E435F0F5A4
:1051CA0083E5822400F582E5833400F583E0C45444
:1051DA00F0440FFD7F02128A0AE5792409F81209C0
:1051EA00AFE41203B1E4FBFA7980784B1202A77B91
:1051FA000A7AD77923784012019EA879120A20A840
:10520A00791209AFE5792404F8120A20E579241302
:10521A00F8E6D39400403BA879E8C0E01209AFE56C
:10522A00792411F8E675F008A4FBE5792412F8EB65
:10523A002625E025E024F0F582E43400F583E0F841
:10524A00A3E0F9A3E0FAA3E0FB1200A9D0E0F81268
:10525A000A20E5792404F81209AFE5792411F8E661
:10526A0075F008A4FBE5792412F8EB2625E025E081
:10527A0024F0F582E43400F583120A2CA879E8C0F8
:10528A00E01209AFECC0E0EDC0E0EEC0E0EFC0E034
:10529A00E5792412F8E625E025E02490F582E43445
:1052AA0000F583E0FCA3E0FDA3E0FEA3E0FF7B6F33
:1052BA007A127983783A12019EC8ECC8C9EDC9CA34
:1052CA00EECACBEFCBD0E0FFD0E0FED0E0FDD0E0DD
:1052DA00FC1202A7D0E0F8120A20E579240FF8E6BA
:1052EA00B47318A879E8C0E01209AFE4FBFA792090
:1052FA0078411202A7D0E0F8120A207F757E787DE5
:10530A000C7C35A8791209C712019EA8791209C71F
:10531A0012019EA8791209C712019EECC0E0EDC0E5
:10532A00E0EEC0E0EFC0E07FFA7EED7D6B7C3AA84C
:10533A00791209C712019EA8791209C712019ED0D3
:10534A00E0FBD0E0FAD0E0F9D0E0F81200ADECC012
:10535A00E0EDC0E0EEC0E0EFC0E07F177ED97D1639
:10536A007C40A8791209C712019ED0E0FBD0E0FA6E
:10537A00D0E0F9D0E0F81200AD7BD37A4D79E2782B
:10538A00411200ADA879120A20A879E8C0E01209F2
:10539A00AF7B337A93798878431200A9D0E0F81268
:1053AA000A20E4FFFE7D207C41A8791209C7120178
:1053BA009EE4FBFAF9783F1200AD1203EFEC1203F8
:1053CA00B1E4FBFA792078411202A7A879120A20DF
:1053DA007F007EC07D797C44A8791209C7120344F4
:1053EA00600B4009A879120A384479F99AE4FFFE59
:1053FA007D487CC3A8791209C71203445009A879C9
:10540A00120A38C479F99AA8791209AFE5792414ED
:10541A00F8CBE6CB08E6FA08E6F91209717F0480B0
:03542A00027F01FD
:07542D00E5792417F579224F
:104A69001579A879EBF61579A879EDF61579A8796C
:084A7900EFF6E57924F4F5796C
:104A8100240DF8E664016003024B0DE579240EF86C
:0C4A9100E6FFE579240F1282D91289FF9C
:104A9D00E579240AF87664E579240AF8E6D39400DA
:104AAD004023E579240BF87603E579240BF8E6D35A
:104ABD009400400900E579240BF81680ECE5792483
:054ACD000AF81680D27A
:104AD200E579240CF8E6B477047D8880027D8C7F2A
:104AE20002128A0AE579240FF8E6FFE579240EF826
:104AF200E675F008A42FF582E435F0F583E582240B
:104B020000F582E5833400F583E4F0E579240DF8BD
:104B1200E664036003024F78E5792410F8E6D39443
:104B22000240057F00024F7AE579240EF8E6FFE5A0
:104B320079240FF8E6FD7B00E5792404F97A001266
:104B42009E88E5792404F8E65401D3940040057F59
:104B520000024F7AE579240FF8E6FDE579240EF894
:104B6200E6FE75F008A42DF582E435F0F583E582C2
:104B72002400F582E5833400F583E0FFE57924051E
:104B8200F8EFF65401FFE5792410F8EF6660057F2F
:104B920000024F7ACFEECF1282DC7B00E579240649
:104BA200127DFCE579240CF8E664776003024C4739
:104BB200E579240FF8E6FFE579240EF8E6FE75F0B4
:104BC20008A42FF582E435F0F583E5822400F5820E
:104BD200E5833400F583E0045401FD75F008EEA48A
:104BE2002FF582E435F0F583E5822400F582E58332
:104BF2003400F583EDF0E579240FF8E6FF75F0084F
:104C0200EEA42FF582E435F0F583E5822400F582E7
:104C1200E5833400F583E070047D8880027D987F0F
:104C220002128A0AE5792406F81209AFE41203B1E6
:104C3200E4FBFA7980784B1202A77B0A7AD779A330
:104C4200783C024CD7E579240FF8E6FFE579240E8B
:104C5200F8E6FE75F008A42FF582E435F0F583E559
:104C6200822400F582E5833400F583E0045401FDDB
:104C720075F008EEA42FF582E435F0F583E5822481
:104C820000F582E5833400F583EDF0E579240FF831
:104C9200E6FF75F008EEA42FF582E435F0F583E522
:104CA200822400F582E5833400F583E0C454F044A5
:104CB2008CFD7F02128A0AE5792406F81209AFE414
:104CC2001203B1E4FBFA7980784B1202A77B0A7ACD
:104CD200D779A3783E12019EA879120A20E5792499
:104CE2000CF8E6FF64756008EF64766003024DD34A
:104CF200A879E8C0E01209AF7B6F7A127983783A1B
:104D02001202A7D0E0F8120A20E579240CF8E6B4E2
:104D12007618A879E8C0E01209AFE4FBFA792078A6
:104D2200411202A7D0E0F8120A207F757E787D0C2E
:104D32007C35A8791209C712019EA8791209C712F7
:104D4200019EA8791209C712019EECC0E0EDC0E0F5
:104D5200EEC0E0EFC0E07FFA7EED7D6B7C3AA87991
:104D62001209C712019EA8791209C712019ED0E04A
:104D7200FBD0E0FAD0E0F9D0E0F81200ADECC0E0F0
:104D8200EDC0E0EEC0E0EFC0E07F177ED97D167C7B
:104D920040A8791209C712019ED0E0FBD0E0FAD0F8
:104DA200E0F9D0E0F81200AD7BD37A4D79E2784198
:104DB2001200ADA879120A20A879E8C0E01209AF62
:104DC2007B337A93798878431200A9D0E0F8024EB7
:104DD200F6E579240CF8E664776003024EF9A879C7
:104DE200E8C0E01209AF7B007A2479747849120195
:104DF2009ED0E0F8120A207F5D7E0B7D237C2CA8DA
:104E0200791209C712019EA8791209C712019EA838
:104E1200791209C712019EA8791209C712019EECE4
:104E2200C0E0EDC0E0EEC0E0EFC0E07F177EEE7DB7
:104E32008B7C32A8791209C712019EA8791209C780
:104E420012019EA8791209C712019EC8ECC8C9EDC9
:104E5200C9CAEECACBEFCBD0E0FFD0E0FED0E0FD76
:104E6200D0E0FC1200A9ECC0E0EDC0E0EEC0E0EF43
:104E7200C0E07F4B7E5F7D047C38A8791209C7129F
:104E8200019EA8791209C712019ED0E0FBD0E0FA78
:104E9200D0E0F9D0E0F81200ADECC0E0EDC0E0EEF9
:104EA200C0E0EFC0E07F4B7E767D6C7C3DA879123E
:104EB20009C712019ED0E0FBD0E0FAD0E0F9D0E0C1
:104EC200F81200AD7B1F7A85796B78BE1200ADA80F
:104ED20079120A20E4FFFEFDFCA8791209C7120329
:104EE200446014A8791209C7E4FFFE7D7A7C44125B
:104EF20002A7A879120A20E4FFFE7DC87C42A879A5
:104F02001209C712019EE4FBFAF9783F1200AD12B2
:104F120003EFEC1203B1E4FBFA79C878421202A75C
:104F2200A879120A207F5C7EFF7D797C44A87912E1
:104F320009C7120344600B4009A879120A38447960
:104F4200FF5CE4FFFE7D207CC1A8791209C7120331
:104F5200445009A879120A38C11FD70AA879120940
:104F6200AFE5792411F8CBE6CB08E6FA08E6F912A8
:084F720009717F0480027F0138
:074F7A00E5792414F579220A
:106D38001579A879EBF61579A879EDF61579A8797A
:086D4800EFF6E57924F5F57979
:106D5000E579240CF8E664016003026DE6E5792428
:0E6D60000DF8E6FFE579240E1282D91289FFA4
:106D6E00E5792409F87664E5792409F8E6D39400E8
:106D7E004023E579240AF87603E579240AF8E6D368
:106D8E009400400900E579240AF81680ECE5792490
:056D9E0009F81680D287
:106DA3007D057F02128A0AE579240EF8E6FFE5796C
:106DB300240DF8E675F008A42FF582E435F0F58389
:106DC300E5822400F582E5833400F583E4F0EF25C2
:106DD300E025E02490F582E43400F583120A513F64
:106DE300800000E579240CF8E664036003026FF089
:106DF300E579240FF8E6D3940740057F00026FF28C
:106E0300E579240DF8E6FFE579240EF8E6FD7B002D
:106E1300E5792404F97A00129E88E5792404F8E6DA
:106E23005401D3940040057F00026FF2E579240EEC
:106E3300F8E6FDE579240DF8E6FE75F008A42DF5D6
:106E430082E435F0F583E5822400F582E58334009E
:106E5300F583E0FFE579240FF8E66F60057F000214
:106E63006FF2CFEECF1282DC7B00E5792405127D31
:106E7300FCE579240EF8E6FFE579240DF8E6FE75C6
:106E8300F008A42FF582E435F0F583E5822400F5BC
:106E930082E5833400F583E0045407FD75F008EEC2
:106EA300A42FF582E435F0F583E5822400F582E52D
:106EB300833400F583EDF0E579240EF8E6FFE579F8
:106EC300240DF8E675F008A42FF582E435F0F58378
:106ED300E5822400F582E5833400F583E0C454F0B1
:106EE3004405FD7F02128A0AE5792405F81209AFE9
:106EF300E41203B1E4FBFA7980784B1202A77B0A10
:106F03007AD779A3783F12019EC8ECC8C9EDC9CAE4
:106F1300EECACBEFCB7F0A7ED77D237C3F1200A93D
:106F2300A879120A20A879E8C0E01209AFE4FBFAB5
:106F3300797A78441202A7D0E0F8120A20A879E8F7
:106F4300C0E01209AF7B007A247974784912019E5C
:106F5300D0E0F8120A20A879E8C0E01209AF7B9AC2
:106F63007A99798878431200A9D0E0F8120A20E4CC
:106F7300FFFE7DC87C42A8791209C712019EE4FB7B
:106F8300FAF9783F1200AD1203EFEC1203B1E4FB00
:106F9300FA79C878421202A7A879120A20E4FFFE00
:106FA3007D167C43A8791209C7120344600B40097C
:106FB300A879120A384479FF5CE4FFFE7D5C7CC249
:106FC300A8791209C71203445009A879120A38C4D0
:106FD30079FF5CA8791209AFE5792410F8CBE6CBE9
:0F6FE30008E6FA08E6F91209717F0480027F01BF
:076FF200E5792413F5792273
:0C9FB4007F01128B5F7FFC129FC07F00BA
:089FC0001579A879EFF6157977
:109FC800C2B3C2B1000000000000000000000000A1
:109FD8000000000000000000A879E4F6A879E6C3B4
:109FE80094085047D2B008E6FF548094004003D349
:109FF8008001C392B30000000000000000000000D0
:10A00800000000000000000000C2B00000000000D6
:10A01800000000000000000000000000000000A890
:10A028007908EF25E0F6A8790680B1D2B1C2B3006D
:10A038000000000000000000000000000000000018
:03A0480000000015
:05A04B000579057922F2
:108B5F001579A879EDF61579A879EFF615791579C4
:108B6F00C2B3C2B10000000000000000000000000E
:108B7F000000000000000000A8790808E62450A8B3
:108B8F007908F6A879E4F6A879E6C394085047D295
:108B9F00B008E6FF548094004003D38001C392B322
:108BAF0000000000000000000000000000000000B6
:108BBF0000000000C2B00000000000000000000034
:108BCF0000000000000000000000A87908EF25E079
:108BDF00F6A8790680B1A8790808E62450A8790884
:108BEF00F6A879E4F6A879E6C394085040D2B0C24B
:108BFF00B3000000000000000000000000000000B3
:108C0F000000000000C2B0000000000000000000E3
:108C1F00000000000000000000000008E8C0E0E6CF
:108C2F0025E0FFD0E0F8EFF6A8790680B8A879E440
:108C3F00F6A879E6C39408504ED2B0E5792403F82C
:108C4F00E6FF5480D394004003D38001C392B30056
:108C5F000000000000000000000000000000000005
:108C6F00000000C2B0000000000000000000000083
:108C7F00000000000000000000E5792403F8EF2554
:108C8F00E0F6A8790680AAD2B1C2B30000000000B6
:0F8C9F00000000000000000000000000000000C6
:078CAE00E5792404F57922A9
:10889900157915791579A879C6EBC608C6EAC60807
:0988A900C6E9C6E57924FCF57965
:1088B200C2B1000000000000000000000000000043
:1088C200000000000000F8087601A879E4F6A87913
:1088D200E6C394085047D2B008E6FF5480940040A3
:1088E20003D38001C392B300000000000000000027
:1088F2000000000000000000000000C2B000000004
:108902000000000000000000000000000000000065
:0D89120000A87908EF25E0F6A8790680B1ED
:10891F00A87908087605A8790808E6D394004022BC
:10892F00E5792403F87613E5792403F8E6D3940068
:10893F00400900E5792403F81680ECA87908081699
:02894F0080D4D2
:10895100A879E4F6E5792404F8CBE6CB08E6FA0831
:10896100E6F9120A8200000000A879E6C3941850C3
:1089710070D2B00000000000000000000000000004
:1089810000000000000000E5792404F8CBE6CB08E4
:10899100E6FA08E6F9120921780112090EC8ECC8B5
:1089A100C9EDC9CAEECACBEFCBA2B4E4334BFFEA9F
:1089B100FEE9FDE8FCE5792404F8CBE6CB08E6FA0C
:1089C10008E6F9120971C2B00000000000000000C1
:1089D100000000000000000000000000A8790680EF
:1089E10088D2B1000000000000000000000000007B
:0789F100000000000000007F
:0789F800E5792407F579225F
:10607D001579A879EBF61579A879EDF61579A87942
:08608D00EFF6E57924F6F57940
:10609500240BF8E66401600302616CE579240CF8D1
:1060A500E6FFE579240D12B31B7D027F00128B5F9D
:1060B5001D7F02128B5F7DD07F03128B5F7FF012F5
:1060C5009FC0E5792404F8120A38000000007FA07B
:1060D5007E867D017C00E5792404F81209C7C31288
:0760E50008FD505730B554CF
:1060EC00E5792408F87601E5792408F8E6D39400DC
:1060FC004023E5792409F87603E5792409F8E6D3F9
:10610C009400400900E5792409F81680ECE579241F
:05611C0008F81680D216
:10612100E5792404F81209AFEF2401FFE43EFEE40F
:106131003DFDE43CFCE5792404F8120A2080937DBE
:106141000F129FB4E579240DF8E6FFE579240CF8E8
:10615100E675F008A42FF582E435F0F583E5822495
:1061610088F582E5833402F583E4F0E579240BF8C0
:10617100E6640360030263F9E579240EF8E6D3943B
:106181000740057F000263FBE579240CF8E6FFE593
:1061910079240D12B31BE5792404F8120A380000A2
:1061A1000000E47F107E27FDFCE5792404F8120944
:0A61B100C7C31208FD505730B55463
:1061BB00E5792408F87601E5792408F8E6D394000C
:1061CB004023E5792409F87603E5792409F8E6D329
:1061DB009400400900E5792409F81680ECE5792450
:0561EB0008F81680D247
:1061F000E5792404F81209AFEF2401FFE43EFEE440
:106200003DFDE43CFCE5792404F8120A208094E486
:106210007F107E27FDFCE5792404F81209C7C3121C
:1062200008FD7004FF0263FBE579240DF8E6FEE546
:1062300079240CF8E675F008A42EF582E435F0F523
:1062400083E5822488F582E5833402F583E0FDE569
:1062500079240EF8E66D60057F000263FBE5792482
:106260000DF8E6FFE579240CF8E6FCED045407FD93
:1062700075F008ECA42FF582E435F0F583E582246F
:1062800088F582E5833402F583EDF075F008ECA41F
:106290002EF582E435F0F583E5822488F582E583E6
:1062A0003402F583E0C454F0440FFD129FB47B0028
:1062B000E5792404F97A00128899E5792404F81222
:1062C00009AF780812090EEC1203B1A879120A205E
:1062D000E4FBFA7980784FE8C0E0A8791209AFD0E2
:1062E000E0F81202A7E4FBFA79A0784012019EA818
:1062F00079120A20E579240AF8E6B46402803FE5C1
:1063000079240AF8E6B4652DE4FBFA79207840E8B0
:10631000C0E0A8791209AFD0E0F81202A7E4FBFAB6
:1063200079A0784112019EE4FBFA792078C112002D
:10633000ADA879803EE579240AF8E6B46617A87915
:10634000E8C0E01209AFE4FBFA7980783F12019EC1
:10635000D0E0F8801EE579240AF8E6B46718A87939
:10636000E8C0E01209AFE4FBFA7920784112019EFF
:10637000D0E0F8120A20E579240AF8E6FF646560A7
:1063800004EFB4672A7F007E407D1C7C46A879120A
:1063900009C712019EE4FBFAF9783F1200AD12031F
:1063A000EFEC1203B17B007A40791C784680287F9D
:1063B000007E507DC37C47A8791209C712019EE474
:1063C000FBFAF9783F1200AD1203EFEC1203B17B38
:1063D000007A5079C378471202A7A879120A20A838
:1063E000791209AFE579240FF8CBE6CB08E6FA0875
:0B63F000E6F91209717F0480027F01B2
:0763FB00E5792412F5792277
:1072AC001579A879EBF61579A879EDF61579A87901
:0872BC00EFF6E57924F5F57900
:1072C400240CF8E66403600302754FE579240FF893
:1072D400E6FED3940340057F000275517401C8EEA5
:1072E400C8088002C333D8FCA8790808F67584015D
:1072F400E5792403F8120A3800000000A879E4F6BE
:10730400A879E6C3940A40030273BCE4F5CCF5CD36
:10731400F5C975C804E579240DF8E6FFE579240E6E
:1073240012B31BE579240DF8E6FFE579240EF8E69F
:10733400FDE4FB12B3207F0012B0ACE579240DF814
:10734400E6FFE579240EF8E6FD7B00A979097A00C9
:10735400129E88A8790808C9E8C9A87908E6576080
:1073640005E5C830E7D0E4F5C8E5792403F8E8C0BA
:10737400E01209AFECC0E0EDC0E0EEC0E0EFC0E029
:10738400AFCDEFFEADCC7C00E42DFFEC3ECBEFCBDC
:10739400FAE4F9F8D0E0FFD0E0FED0E0FDD0E0FC64
:1073A400EF2BFFEE3AFEE93DFDE83CFCD0E0F8129D
:1073B4000A20A87906027304E5C85480FFBF012798
:1073C400E579240BF8E6B4700FE5792407F8120A7E
:1073D40038411FFFFF027532E5792407F8120A3895
:1073E4004479FFFE027532E5792403F81209AFE40B
:1073F4001203B1ECC0E0EDC0E0EEC0E0EFC0E0A8E5
:1074040079E6FCE41203BBC8ECC8C9EDC9CAEECAEC
:10741400CBEFCBD0E0FFD0E0FED0E0FDD0E0FC121B
:1074240002A7E4FBFA79C478421202A7E4FBFA79D2
:1074340040784112019EE5792407F8120A20E57983
:107444002407F8E8C0E01209AF7B007A2479747845
:10745400491202A7D0E0F8120A20E579240BF8E6D5
:1074640064707BCD7ACC798C783F7044E8C0E0E5D9
:10747400792407F81209AFD0E0F81202A77B007A4A
:10748400B8790878491202A77B287A6B796E784E0E
:1074940012019EE5792407F8120A20E5792407F8F9
:1074A400E8C0E01209AF7B777ABE799F783D8041CE
:1074B400E8C0E0E5792407F81209AFD0E0F8120239
:1074C400A7E4FBFA79AF78451202A77B287A6B7997
:1074D4006E784E12019EE5792407F8120A20E579A8
:1074E4002407F8E8C0E01209AF7B9A7A9979F97811
:1074F400401200A9D0E0F8120A20E4FFFE7D7A7C55
:1075040044E5792407F81209C712019EE4FBFAF94D
:10751400783F1200AD1203EFEC1203B1E4FBFA79E9
:107524007A78441202A7E5792407F8120A20E5794B
:107534002407F81209AFE5792410F8CBE6CB08E666
:0D754400FA08E6F91209717F0480027F0148
:07755100E5792413F579220E
:1016C0001579A879EBF61579A879EDF61579A87949
:0816D000EFF6E57924F0F5794D
:1016D800E5792412F8E675F008A4FFE5792413F8F3
:1016E800EF26FFE579240DF8EFF6E5792411F8E601
:1016F80064046003021818E5792414F8E67032E5EA
:1017080079240DF8E625E025E02450F582E434013B
:10171800F583120A5142960000E5792415F8CBE6C4
:10172800CB08E6FA08E6F9120A8242960000021887
:1017380013E5792414F8E6B40132E579240DF8E6C6
:1017480025E025E02430F582E43403F583120A51BC
:1017580000000000E5792415F8CBE6CB08E6FA0886
:10176800E6F9120A8200000000021813E579241431
:10177800F8E6B40231E579240DF8E625E025E02401
:10178800B0F582E43401F583120A513F800000E588
:10179800792415F8CBE6CB08E6FA08E6F9120A82AE
:1017A8003F8000008065E5792414F8E6FFB4032B38
:1017B800E579240DF8E625E02458F582E43402F5AD
:1017C80083E4F0A3743CF0E5792415F8CBE6CB0864
:1017D800E6FA08E6F9E475F03C802DEFB4042CE550
:1017E80079240DF8E625E024A8F582E43406F5838B
:1017F800E4F0A37405F0E5792415F8CBE6CB08E608
:10180800FA08E6F9E475F0051208BA7F0002202903
:10181800E579240DF8E624D8F582E43406F583E06A
:1018280060030218EF12B362E579240DF8E625E0AB
:1018380025E024A0F582E43402F583E0F8A3E0F97A
:10184800A3E0FAA3E0FBC3EF9BFFEE9AFEED99FD40
:10185800EC98FCECC0E0EDC0E0EEC0E0EFC0E0E5E5
:1018680079240DF8E625E02458F582E43402F5835E
:10187800E0FEA3E0FF7C007D64120782CBEFCBCAB9
:10188800EECAE4F9F8D0E0FFD0E0FED0E0FDD0E009
:10189800FCC31208FD40030219CBE579240DF8E6D4
:1018A80024D8F582E43406F5837401F012B362E5B6
:1018B80079240DF8E6FB25E025E024A0F582E43440
:1018C80002F583120A2CEB25E025E02450F582E48A
:1018D8003401F583E0FCA3E0FDA3E0FEA3E0FFA84C
:1018E80079120A2002199412B362E579240DF8E6F8
:1018F80025E025E024A0F582E43402F583E0F8A38E
:10190800E0F9A3E0FAA3E0FBC3EF9BFFEE9AFEED3C
:1019180099FDEC98FCECC0E0EDC0E0EEC0E0EFC053
:10192800E0E579240DF8E625E024A8F582E43406FC
:10193800F583E0FEA3E0FF7C007D64120782CBEF15
:10194800CBCAEECAE4F9F8D0E0FFD0E0FED0E0FD63
:10195800D0E0FCC31208FD506AE579240DF8E624AE
:10196800D8F582E43406F583E4F012B362E579240D
:101978000DF8E625E025E024A0F582E43402F5839D
:10198800120A2CA879120A3800000000A9791579E2
:1019980015791579A879760008760008C6E9C6157C
:1019A80079A879E4F6E5792417F8E61579A879F69F
:1019B800E5792417F8E6FB7D02E5792415F8E6FFBA
:1019C8001216C0E5792411F8E664016003021A6B67
:1019D800E5792412F8E6FFE5792413F8E6FD7B0E95
:1019E80012A335E5792412F8E6FFE5792413F8E621
:0C19F800FD7B0E129D511282CE1289FF61
:101A0400E579240EF87664E579240EF8E6D394009B
:101A14004023E579240FF87603E579240FF8E6D31B
:101A24009400400900E579240FF81680ECE5792448
:051A34000EF81680D23F
:101A39007D077F02128A0AE579240DF8E624D8F594
:101A490082E43406F5837401F012B362E579240D5A
:101A5900F8E625E025E024A0F582E43402F58312B6
:101A69000A2CE5792411F8E664026003021D41E5B8
:101A7900792414F8E6703FE5792415F8CBE6CB080C
:101A8900E6FA08E6F9120921E4FBFAF9F812034427
:101A99005024E5792415F8CBE6CB08E6FA08E6F9EF
:101AA900120921E579240DF8E625E025E02450F511
:101AB90082E434018058E5792414F8E6B40124E578
:101AC900792415F8CBE6CB08E6FA08E6F9120921DC
:101AD900E579240DF8E625E025E02430F582E434A3
:101AE90003802BE5792414F8E6B40229E579241555
:101AF900F8CBE6CB08E6FA08E6F9120921E57924DC
:101B09000DF8E625E025E024B0F582E43401F583FB
:101B1900120A2C8062E5792414F8E6FFB4032BE558
:101B2900792415F8CBE6CB08E6FA08E6F912081F7E
:101B3900FDE579240DF8E625E02458F582E4340220
:101B4900F583E5F0F0A3EDF0802DEFB40429E579F4
:101B59002415F8CBE6CB08E6FA08E6F912081FFFC8
:101B6900E579240DF8E625E024A8F582E43406F5A4
:101B790083E5F0F0A3EFF0E5792414F8E6D39400B7
:101B890040057F00022029E5792415F8CBE6CB082A
:101B9900E6FA08E6F9120921A879120A20E4FFFEFB
:101BA900FDFCA8791209C71203445009A879120A41
:101BB9003800000000E4FFFE7DC87C42A8791209C4
:101BC900C7120344600B4009A879120A3842C800B9
:101BD90000E4FBFA79C87842E8C0E0A8791209AFB5
:101BE900D0E0F81202A77B007AFF797F78471201CB
:101BF9009E1203EFE579240AF8EEF608EFF6E57987
:101C09002412F8E6FFE5792413F8E6FDE4FB129DBA
:101C190051E579240CF8E4F6E579240CF8E6FFC3DC
:101C290094045033EF940140047F0480027F001232
:101C39009D35E5792412F8E6FFE5792413F8E6FDE8
:101C4900E5792405F8E64408FB129D51129D3CE50F
:101C590079240CF80680C1E579240CF8E4F6E579D5
:101C6900240CF8E6C39404504DE5792414F8E6549D
:101C790008D3940040047F0480027F00129D35E55B
:101C8900792412F8E6FFE5792413F8E6FDE57924CD
:101C990005F8E64408FB129D51129D3CE579241490
:101CA900F8E8C0E0E625E0FFD0E0F8EFF6E57924B2
:101CB9000CF806021C67E579240CF8E4F6E57924AA
:101CC9000CF8E6C39410505DE579240AF8E65480CF
:101CD900FED3E49400EE940040047F0480027F0068
:101CE900129D35E5792412F8E6FFE5792413F8E623
:101CF900FDE5792405F8E64408FB129D51129D3C47
:101D0900E579240AF8E8C0E0C9E8C909E725E0FF50
:101D190019E733FED0E0F8EEF608EFF6E579240C82
:101D2900F806021CC6E5792412F8E6FFE5792413C2
:101D3900F8E6FD7B0E129D51E5792411F8E664035E
:101D49006003022027E5792414F8E67013E5792465
:101D59000DF8E625E025E02450F582E434018036CB
:101D6900E5792414F8E6B40113E579240DF8E6259C
:101D7900E025E02430F582E43403801AE57924145F
:101D8900F8E6B40221E579240DF8E625E025E024FA
:101D9900B0F582E43401F583E0FCA3E0FDA3E0FEA5
:101DA900A3E0FF02200EE5792414F8E6FEB4032827
:101DB900E579240DF8E625E02458F582E43402F5A6
:101DC90083E0F9A3E0FDE5792415F8CBE6CB08E635
:101DD900FA08E6C98DF0802AEEB4042EE579240DBF
:101DE900F8E625E024A8F582E43406F583E0F9A3B2
:101DF900E0FFE5792415F8CBE6CB08E6FA08E6C951
:101E09008FF01208BA7F02022029E5792414F8E636
:101E1900640560057F00022029E5792412F8E6FFB0
:101E2900E5792413F8E6FD7B00E5792404F97A00C5
:101E3900129E88E5792404F8E65401D394004005FC
:101E49007F000220291282CE7B00E5792406127DCB
:101E5900FC7D077F02128A0AE5792406F81209AF88
:101E6900E41203B1E4FBFA7980784B1202A77B0AEA
:101E79007AD779A3784012019E7B0A7AD779237899
:101E8900C01200ADA879120A20A879E8C0E01209A9
:101E9900AF7B387A1F7943784112019ED0E0F8125E
:101EA9000A20A879E8C0E01209AFECC0E0EDC0E073
:101EB900EEC0E0EFC0E0E579240DF8E625E025E085
:101EC9002450F582E43401F583E0FCA3E0FDA3E0AE
:101ED900FEA3E0FFE4FBFA797A78441202A7C8EC82
:101EE900C8C9EDC9CAEECACBEFCBD0E0FFD0E0FE3E
:101EF900D0E0FDD0E0FC1202A7D0E0F8120A207B66
:101F0900CD7ACC792C7840E8C0E0A8791209AFD015
:101F1900E0F81202A7C8ECC8C9EDC9CAEECACBEFEE
:101F2900CBE4FFFE7DC87C421200A9A879120A20E1
:101F3900E579240DF8E625E025E02430F582E4343E
:101F490003F583E0F8A3E0F9A3E0FAA3E0FBE8C016
:101F5900E0A8791209AFD0E0F81200A9E579240DBB
:101F6900F8E625E025E024B0F582E43401F583E0C4
:101F7900F8A3E0F9A3E0FAA3E0FB12019EA8791205
:101F89000A207F007E507DC37C47A8791209C712B9
:101F9900019EE4FBFAF9783F1200AD1203EFEC124F
:101FA90003B17B007A5079C378471202A7A8791246
:101FB9000A20E579240DF8E624D8F582E43406F5FB
:101FC90083E06401705412B362E579240DF8E625C3
:101FD900E025E024A0F582E43402F583E0F8A3E0EB
:101FE900F9A3E0FAA3E0FBC3EF9BFFEE9AFEED999C
:101FF900FDEC98FCE47B64FAF9F8C31208FD501A69
:10200900A8791209AFE5792415F8CBE6CB08E6FAE9
:1020190008E6F91209717F0480067F0080027F01BA
:07202900E5792418F5792286
:107558001579A879EBF61579A879EDF61579A87952
:08756800EFF6E57924F5F57951
:10757000E579240CF8E664017021E579240DF8E63C
:10758000FFE579240EF8E6FD7BFF129D51E5792495
:107590000DF8E6FFE579240E12A330E579240CF806
:1075A000E6640360030277F1E579240FF8E67012D0
:1075B000E579240DF8E6FFE579240EF8E6FD7BFE7B
:1075C0008010E579240DF8E6FFE579240EF8E6FD54
:1075D0007BFD129D51E579240DF8E6FFE579240E37
:0375E00012B31BC8
:1075E300E5792409F8760AE5792409F8E6D39400C5
:1075F3004023E579240AF87603E579240AF8E6D3EB
:107603009400400900E579240AF81680ECE5792412
:0576130009F81680D209
:1076180030B418E579240DF8E6FFE579240EF8E68C
:10762800FD7BFF129D517F000277F3E5792404F872
:10763800120A3800000000E5792408F8E4F6E57934
:107648002408F8E6C3941B507500000000000000F1
:1076580000000000000000000000000000D2B000A0
:107668000000000000000000000000000000000012
:10767800000000C2B0000000000000000000000090
:10768800000000000000000000E5792404F8120959
:10769800AF780112090EC8ECC8C9EDC9CAEECACB49
:1076A800EFCBA2B4E4334BFFEAFEE9FDE8FCE57951
:1076B8002404F8120A20E5792408F8068080E57980
:1076C800240DF8E6FFE579240EF8E6FD7BFF129D10
:1076D80051E5792404F81209AFE4FFFEFDEC5402E9
:1076E800FC601EE5792404F81209AFE4FFFEFDEC06
:1076F8005401FC600CA879120A3840200000027777
:107708008EE5792404F81209AFE4FFFEFDEC54027B
:10771800FCE4FBFAF9F8C31208FD701DE5792404AE
:10772800F81209AFE4FFFEFDEC5401FC600BA879E8
:10773800120A3800000000804DE5792404F8120987
:10774800AFE4FFFEFDEC5402FCE4FBFAF9F8C312C7
:1077580008FD700CE5792404F81209AF74FF80095C
:10776800E5792404F81209AFE4FC1203B1E4FBFA4A
:107778007980784B1202A7E4FBFA7920784012014D
:107788009EA879120A20E4FFFEFD7C41A87912091F
:10779800C712019EE4FBFA792078C11200ADA879DE
:1077A800120A207F007E247D747C49A8791209C7BB
:1077B80012019EE4FBFAF9783F1200AD129C857B1A
:1077C800007A24797478491202A7A879120A20A8A5
:1077D800791209AFE5792410F8CBE6CB08E6FA0868
:0B77E800E6F91209717F0480027F00A7
:0777F300E5792413F579226A
:067F9D008F448D458B4668
:107FA300E4FFFEFDFCAB4AAA49A948A847120344D3
:107FB3005009E4F54AF549F548F547E4FFFE7D48E5
:107FC3007C43AB4AAA49A948A847120344600D4021
:107FD3000BE4F54AF549754848754743AF4AAE493E
:107FE300AD48AC47ECC0E0EDC0E0EEC0E0EFC0E070
:107FF300E54575F008A47C002546FFEC35F0FEEF5F
:108003007802C333CE33CED8F924A8F58274033E65
:10801300F583D0E0FFD0E0FED0E0FDD0E0FC120A13
:108023002CE4FBFA79907842AF4AAE49AD48AC47AD
:108033001202A7E4FBFA792078401202A77B007AA8
:10804300FF797F784712019E1203EF8E4B8F4C7B93
:1080530048AD45AF44129D517B06AD45AF4412B3C5
:1080630020E4FDEDD394014003D38001C392B30018
:1080730000000000000000000000000000000000FD
:10808300000000D2B000000000000000000000006B
:10809300000000000000000000C2B00DBD04C4E4F5
:1080A300FDE5465408D394004003D38001C392B343
:1080B30000000000000000000000000000000000BD
:1080C30000000000D2B0000000000000000000002B
:1080D30000000000000000000000C2B0E54625E0FB
:1080E300F5460DBD04BBE4FDE54B5480FED3E4949B
:1080F30000EE94004003D38001C392B3000000005C
:10810300000000000000000000000000000000006C
:10811300D2B00000000000000000000000000000DA
:10812300000000000000C2B0E54C25E0F54CE54B33
:1081330033F54B0DBD10B17B40AD45AF44029D51AE
:103EF0001579A879EBF61579A879EDF61579A879F1
:083F0000EFF6E57924F0F579F4
:103F0800E5792412F8E6FF75F008A4FEE579241394
:103F1800F8E6FD2EFEE579240DF8EEF6E579241194
:103F2800F8E664016003023FFF7B7812A335E57968
:103F38002412F8E6FFE5792413F8E6FD7B40129D8C
:103F480051E5792412F8E6FFE5792413F8E6FD7BBC
:103F580070129D51E5792412F8E6FFE579241312D1
:0C3F6800B31B1289FF7D117F07128A0A2B
:103F7400E579240EF87664E579240EF8E6D3940006
:103F84004023E579240FF87603E579240FF8E6D386
:103F94009400400900E579240FF81680ECE57924B3
:053FA4000EF81680D2AA
:103FA9007D577F02128A0AE5792413F8E6FEE5793E
:103FB9002412F8E6FF75F008A42EF582E435F0F531
:103FC90083E5822400F582E5833403F583E4F07503
:103FD900F008EFA42EF582E435F0F583E582241884
:103FE900F582E5833403F583E4F0E5792413F8E6F3
:103FF900FD7B40129D51E5792411F8E664026003C6
:10400900024091E5792414F8E6FED3940740057F30
:1040190000024501EE7029E5792415F8CBE6CB08B5
:10402900E6FA08E6F9E5792413F8E675F003A4241D
:1040390030F582E43400F583EBF0A3EAF0A3E9F06C
:10404900E5792415F8CBE6CB08E6FA08E6F9120972
:1040590021A879120A20A8791209AFE5792413F861
:10406900E675F003A42430F582E43400F583E0FB1F
:10407900A3E0FAA3E0F9E5792414F8E675F004A4BD
:10408900F58285F08312098BE5792411F8E664033A
:1040990060030244FFE5792414F8E6FFC39408405D
:1040A90006EFD3941740057F00024501E5792412F4
:1040B900F8E6FFE5792413129E7CE5792408F8E6F1
:1040C90030E003024300E5792413F8E6FDE579249D
:1040D90012F8E6FE75F008A42DF582E435F0F583B3
:1040E900E5822400F582E5833403F583E02408FBA7
:1040F900E433FAE5792414F8E66B7001EA60057F88
:1041090000024501CFEECF7B50129D511282CE1293
:104119007DF6E5792413F8E6FFE5792412F8E6FE41
:1041290075F008A42FF582E435F0F583E5822400C3
:10413900F582E5833403F583E0045407FD75F0083F
:10414900EEA42FF582E435F0F583E5822400F582AB
:10415900E5833403F583EDF0E5792413F8E6FFE50B
:10416900792412F8E675F008A42FF582E435F0F504
:1041790083E5822400F582E5833403F583E09038F2
:104189002493C454F04407FD7F02128A0AE5792476
:1041990012F8E6FFE5792413F8E6FD7B40129D51FC
:1041A900E5792409F81209AFE41203B1E4FBFA79BD
:1041B90080784B1202A77B0A7AD779A3784012013B
:1041C9009E7B0A7AD7792378C01200ADA879120AA2
:1041D90020A879E8C0E01209AFE4FBFA79C878426F
:1041E90012019ED0E0F8120A20E4FFFE7D7A7C4499
:1041F900A8791209C712019EE4FBFAF9783F120067
:10420900AD1203EFEC1203B1E4FBFA797A784412A8
:1042190002A7A879120A20A8791209AFE57924150D
:10422900F8CBE6CB08E6FA08E6F9120971E5792434
:1042390013F8E675F003A42430F582E43400F5831D
:10424900E0FBA3E0FAA3E0F9E5792414F8E675F0B8
:1042590004A4FFE92FF9EA35F0FA90FFE01209F01A
:10426900E8C0E0A8791209AFD0E0F81200A9E57911
:104279002404F8120A20E5792404F81209AF12B3CC
:10428900C77BA67A9B7944783B1203445064E5794D
:104299002413F8E675F008A4FFE5792414F8E67C00
:1042A900002FFFEC35F0FEEF7802C333CE33CED8C2
:1042B900F92488F58274033EF583E0FCA3E0FDA3AD
:1042C900E0FEA3E0FFE5792404F81209C71200A96A
:1042D9008F4A8E498D488C47E5792412F8E6FFE527
:1042E900792413F8E6FDE5792414F8E624F8FB129D
:1042F9007F9D7F04024501E5792408F8E630E10352
:104309000244FBE5792413F8E6FDE5792412F8E681
:10431900FE75F008A42DF582E435F0F583E58224D5
:1043290018F582E5833403F583E02410FBE433FABE
:10433900E5792414F8E66B7001EA60057F0002450F
:1043490001CFEECF7B60129D511282CE127DF6E530
:10435900792413F8E6FFE5792412F8E6FE75F008EA
:10436900A42FF582E435F0F583E5822418F582E57A
:10437900833403F583E0045407FD75F008EEA42F98
:10438900F582E435F0F583E5822418F582E5833476
:1043990003F583EDF0E5792413F8E6FFE5792412B6
:1043A900F8E675F008A42FF582E435F0F583E58287
:1043B9002418F582E5833403F583E090382C93C4FF
:1043C90054F04407FD7F02128A0AE5792412F8E6BF
:1043D900FFE5792413F8E6FD7B40129D51E5792428
:1043E90009F81209AFE41203B1E4FBFA7980784BBA
:1043F9001202A77B0A7AD779A3784012019E7B0A19
:104409007AD7792378C01200ADA879120A207B00E7
:104419007A40791C7846E8C0E0A8791209AFD0E063
:10442900F81202A77B007A247974784912019EA8B0
:1044390079120A20E4FFFE7D7A7C44A8791209C723
:1044490012019EE4FBFAF9783F1200AD1203EFEC7A
:104459001203B1E4FBFA797A78441202A7A8791217
:104469000A20E5792414F8E6B41029E5792415F829
:10447900CBE6CB08E6FA08E6F9E5792413F8E67500
:10448900F003A42410F582E43402F583EBF0A3EAE7
:10449900F0A3E9F0A8791209AFEEC0E0EFC0E0E5BA
:1044A900792413F8E675F003A42410F582E43402A4
:1044B900F583E0FBA3E0FAA3E0F9E5792414F8E633
:1044C90075F004A4FFE92FF9EA35F0FA90FFC0D09E
:1044D900E0FFD0E0FE12098BA8791209AFE5792433
:1044E90015F8CBE6CB08E6FA08E6F91209717F045C
:0844F90080067F0080027F01B4
:07450100E5792418F5792289
:10B0D80020202020557067726164696E6700202007
:10B0E80020204669726D776172652E2E2E002452DB
:0BB0F80065763A20353032322024000B
:0FADC9000184FF420700FFFF440708000000005D
:10640200E47880F612B388C28575840F75E104E4DE
:10641200F5E275E344F58475B7B075840F758A8328
:10642200F597438901758D01758F01758E04F542CB
:10643200F5430543E54370020542640F454270F29D
:10644200438902E4F542F543AE42AF43E4FCFD7BEF
:10645200507AC3F9F8D31208E7400FE58920E40A1D
:106462000543E54370E2054280DE75970212A6D429
:1064720012A88F8F41E4F584E541D39400400EE5E4
:10648200EF5402D394004005AF411285BF12B1C947
:10649200E4FF12B1E843EF04E4F542F5437D01AFB6
:1064A2004312B0520543E54370020542C39402E52C
:1064B20042940040E8E4F520C22AC228C22EC22D2E
:1064C200C22C7880F6C22F08F67886F618F6788BFA
:1064D200F6F542F54374102543F582E43407F5835B
:1064E200E4F00543E54370020542B400E8E542B436
:1064F20001E3E4F542F54374102543F582E43408E0
:10650200F583E4F00543E5437002054264404542E9
:1065120070E5E4F584E5EF20E10CE5EF5408D3944F
:10652200004003D38001C392037D08E4FF12AC82D2
:106532007D087F0112AC82127A3FE4788AF6788273
:10654200F6AB15AA16A9177882E6FF75F020A4F516
:106552008285F083120721FE788A26F6EE6005789E
:10656200820680DDEFD394004032AB15AA16A9173C
:1065720090000D120AAC120708F541745512074E2D
:1065820012070864556002D22C74AA12074E120731
:106592000864AA6002D22CE54112074EE4F584E5B4
:1065A200EF5402D3940040047F018002E4FF12966C
:1065B200CA8F40E54020E036C22974FF788DF60884
:1065C200F608F608F67E007F107D007B007A0079DF
:1065D20093120B2F7548FF75493A754A6E754B0039
:1065E200754C107B007A00799312ABDF8002D229BE
:1065F20090B0FDE493FF3395E0FEEF24D0FFEE343C
:10660200FFFE7C007D64120782AA06AB0790B0FCF5
:10661200E493FF3395E0FEEF24D0FFEE34FFFE7CDF
:10662200037DE8120782EF2BFBEE3AFA90B0FEE40C
:1066320093FF3395E0FEEF24D0FFEE34FFFE7C00A3
:106642007D0A120782EF2BFFEE3AFEA3E493FD339D
:1066520095E0FCED24D0FDEC34FFCD2F7892F6EDE1
:106662003E18F6E54030E103026710E4F542F543D7
:10667200E543AE427805C333CE33CED8F9FFAB152E
:10668200AA16A917F5828E831207216078E92FF9DD
:10669200EA3EFA90000412072120E25EE4F53FE5AB
:1066A2003FC3787F965053E543AE427805C333CE5D
:1066B20033CED8F9AB15AA16A917F5828E83120725
:1066C20021FF7E00C006C0077D00E543AE4278058B
:1066D200C333CE33CED8F929F9EA3EFA90000D122F
:1066E2000AAC788AE6853FF0A429F9EA35F0FAD0B7
:1066F20007D006120B2F053F80A50543E543700224
:1067020005420266727F01128143C22B8007E4FFB9
:10671200128143D22BE4F542F5437A007B967D0346
:10672200AF4312A20F0543E54370020542C3940230
:06673200E542940040E482
:01673800223E
:05B3E700788BE6FF2257
:03002300029195B2
:10919500C0E0C0F0C083C082C0D075D000C000C0A0
:1091A50001C002C003C004C005C006C00730993E17
:1091B500C2997886067986E77881667015F678868D
:0191C500F6B3
:0D91C60075270A75281300D528FCD527F65B
:0491D300C285801CB5
:0D91D70075271475281300D528FCD527F640
:1091E4007886E62410F582E43408F583E0F59920C6
:1091F4009803029290209A08202A05C29802928C21
:10920400C29A7885E6062410F582E43407F583E5EE
:1092140099F0C298E6FFB40112900710E0FE7003C3
:10922400F68069EE54072402788CF6EFB4020D78C8
:109234008CE6B40907900711E02403F67885E6FF6D
:10924400B40007E4B40103F68042EFC3788C96407F
:109254003B7885E624FFFDE434FFFC7B017A077943
:109264001012A3BD7885E6240FF582E43407F58354
:08927400E06F60047600801435
:0D927C0075271475281300D528FCD527F69A
:1092890012203078857600D007D006D005D004D0DA
:1092990003D002D001D000D0D0D082D083D0F0D07A
:0292A900E032B1
:10002600900711E075F020A4AB152517F9E51635F4
:10003600F0FA90000D120AAC788BE6FF18E68FF006
:10004600A4252BF582E435F0F583120721FF7B000A
:040056007A0079298A
:10005A008F398B3A8A3B893CE4F584EA494B601C28
:10006A00AB3AAA3BA93C120708FFE539FD7C00120E
:0C007A00B3D4AB3AAA3BA93CEF12074EEE
:0D008600753D14753E1300D53EFCD53DF6CA
:0E0093008539997F0112B0AC3099FDC29922D7
:10AF8D009008107478F07885E6240FF582E4340784
:09AF9D00F583E0900811F07F0239
:09AFA600E4F5847881EFF6D28510
:0DAFAF00753914753A1300D53AFCD539F602
:07AFBC00900810E0F5992256
:10AE5400C9EFC9E964017028EDC39B4034787FE6EB
:10AE6400FFEB2FFFE433FEEDC39FEE6480F87480A4
:10AE740098501ED22AC3ED9B788BF67887760122F0
:10AE8400B90214ED6B700AD22A788BF678877602B1
:08AE940022C22AE47887F622AD
:10A9CB00C9EFC9BAFF15BBFF12ED6B7002EC6A70D1
:10A9DB0049D22A788BF67887E9F622E9640170254B
:10A9EB00C3ED9BEC9A401C787FE62BFFE43AFEC349
:10A9FB00ED9FEC9E500DD22AC3ED9B788BF678879A
:10AA0B007601228015B90218ED6B7002EC6A700AA0
:10AA1B00D22A788BF67887760222C22AE47887F6D8
:01AA2B002208
:10203000900710E0FF54F8F52AE4F584EF120ADC6B
:10204000208009208D0A20A01020A91120BA12207A
:10205000D11920E71A210C2021152821B12922B3FA
:102060003322EE37231E39233841234349234E4E72
:1020700023815023C961227D7023C198000023F978
:10208000900711E0FD788EE6FB7F01802790071115
:10209000E0FCA3E0FD788DE6FA08E6FB7F01802BEB
:1020A000D22A788776030223F9900711E0FD789011
:1020B000E6FB7F0212AE540223F9900711E0FCA365
:1020C000E0FD788FE6FA08E6FB7F0212A9CB022337
:1020D000F9900711E0FD788EE6FB7F0112AE5420E7
:1020E0002A030223F9801A900711E0FCA3E0FD788F
:1020F0008DE6FA08E6FB7F0112A9CB202A03022312
:10210000F99008107478F07F010223F6E4F58475E5
:10211000EF100223F9C2ACE4F529D285FB7A0079ED
:10212000297F7F12005A7B007A0079297F1E1200D6
:102130005A7B007A0079297F0512005A7882E612CC
:102140000053788DE6120053788EE6120053788F94
:10215000E61200537890E61200537891E61200538D
:102160007892E6120053E4F52B7493252BF8E612CF
:102170000053052BE52BC3941040EEE4F52B74FAC5
:10218000252BF582E43406F583E0120053052BE598
:102190002BC3940640E87B007A007900AF29120037
:0121A0005AE4
:0D21A10075370A75381300D538FCD537F6B0
:1021AE00022268900711E0FFC37882964003022254
:1021BE006FEF75F020A42517F9E51635F085153467
:1021CE00F5358936C2ACE4F529D285FB7A0079293A
:1021DE007F7F12005A7B007A0079297F0D12005AF8
:1021EE00AB34AA35A936120708120053AB34AA3500
:1021FE00A936900001120050AB34AA35A9369000D2
:10220E0002120050AB34AA35A936900003120050CA
:10221E00AB34AA35A936900004120050E4F52BAB6E
:10222E0034E5362405F9E43535FA7E00E9252BF937
:10223E00EE3AFA120708120053052BE52BC3940849
:0D224E0040DD7B007A007900AF2912005AB4
:0D225B0075370A75381300D538FCD537F6F5
:10226800C285D2AC0223F99008107478F0E4A3F088
:102278007F020223F612B37578A3120A2090081081
:10228800747CF078A3E6A3F008E6A3F008E6A3F0D0
:1022980008E6A3F07C007D057B017A08791012A37B
:1022A800BD900815EFF07F060223F6900711E0FFB6
:1022B800B4010FA3E0FDA3E0788DCDF608EDF6029A
:1022C80023C1EFB4020A900712E0788DF60223C109
:1022D800900711E0B4030CA3E0FFA3E0788FCFF6DA
:1022E80008EFF60223C1E4F52B900711E0FFE52B78
:1022F800C39F501B7412252BF582E43407F583E045
:10230800FF7493252BF8EFF6052BE52BB410DAE4D0
:1023180078A2F60223C17A007B327D01788BE6FF32
:1023280012A20F900711E0FDE4FF12AC820223F91C
:10233800900711E024FF92020223F9900711E0248C
:10234800FF92010223F97A007B327D017F0012A2FD
:102358000FE4F52B7411252BF582E43407F583E09F
:10236800FF7402252BF582E43407F583EFF0052B83
:10237800E52BB406DFD22F8078788BE66005752DC3
:1023880002800B202D05752D038003752D01900803
:10239800107479F0A3E52DF07C007D027B017A08AA
:1023A800791012A3BD900812EFF07F0312AFA6E5D3
:1023B8002D6401703CD22E8002D228788076F1807C
:1023C800307A007B327D017F0012A20F90081074D2
:1023D80079F0900711E0900811F07C007D027B01F4
:1023E8007A08791012A3BD900812EFF07F0312AF9C
:1023F800A6E52A64A06003022608900710E064A1FD
:1024080060030224F8A3E0C378829640030224ED17
:10241800AB15AA16A917E0FF75F020A4F58285F080
:1024280083120721F52DEF75F020A429F9EA35F07C
:10243800FA90000412072130E237900711E012B336
:10244800EC8F2D900810747FF0A3E52DF02402FD89
:10245800E433FC7B017A08791012A3BD7412252D90
:10246800F582E43408F583EFF0E52D2403FF022616
:1024780005900711E0FF12B3ECC2ACE4F529D28550
:10248800E52DD39406402B7B007A0079297F7F12B3
:10249800005A7B007A007929AF2D12005AE4F52BF7
:1024A800E52BC3952D5007120026052B80F2052D2C
:1024B8008018E52D2478120053E4F52BE52BC395FD
:1024C8002D5007120026052B80F27B007A00790038
:0524D800AF2912005ABB
:0D24DD0075370A75381300D538FCD537F671
:1024EA000225F79008107478F07F010226059007FC
:1024FA0010E064A260030226087882E6FFA3E0FEE9
:10250A00C39F40030225FDA3E0FDC39F40030225AC
:10251A00FDEE9D40030225FD900711E0F52BE4F541
:10252A0032F533900712E0FFE52BD39F5026AF2BED
:10253A0012B3ECAB15AA16A91775F020E52BA4F572
:10254A008285F0831207212533F533E43532F532DB
:10255A00052B80CFC2ACE4F529D285FB7A00792914
:10256A007F7F12005AC3E5339480E532940050020B
:10257A008007E5324480120053AF331200549007AB
:10258A0011E0F52B900712E0FFE52BD39F5046E4AC
:10259A00F52CAB15AA16A91775F020E52BA4F58220
:1025AA0085F083120721FFE52CC39F5024E52B7584
:1025BA00F020A429F9EA35F0FA90000D120AAC7855
:1025CA008BE6FF18E68FF0A4252C120049052C8013
:1025DA00C1052B80AF7B007A007900AF2912005A1F
:0D25EA0075370A75381300D538FCD537F663
:1025F700C285D2AC800B9008107478F07F0112AFBF
:10260700A6E52A6458704DFA7B327D01788BE6FF88
:1026170012A20F753C01753D08753E117B017A07C3
:10262700791112B07F8F2DE52D2478900810F0EFE7
:102637002401FDE433FC7B017A08791012A3BD74F1
:1026470011252DF582E43408F583EFF0E52D2402FA
:10265700FF12AFA6E52A64806009E52A6488600353
:1026670002282D7887E6B4010F7A007B327D017846
:102677008BE6FF12A20F801AE4F52BE52BC3787FB8
:1026870096500F7A007B327D01AF2B12A20F052BDC
:1026970080E9900710E05407F52DB4070A752C015F
:1026A700A3E0F52DA38006E4F52C900711E0F52EA5
:1026B700152DE52EC3788296400302281AAB15AA7A
:1026C70016A91775F020E52EA4F58285F083120769
:1026D70021FFE52DD39F40028F2D7887E6B40109AE
:1026E700788BE6F531F5308009E4F530787FE6142C
:1026F700F531788BA630788BE6D3953140030227E6
:10270700F1E4F52BE52BC3952D40030227E6E52ED3
:1027170075F020A4AB152517F9E51635F0FA9000EA
:102727000412072130E2030227E19000011207217A
:1027370064387041E52DD394044011E52C252B24F2
:1027470012F582E43407F583E0FD80707885E6C3EF
:10275700952BFFE49400FE740E2FF58274073EF567
:1027670083E0FDE52E75F020A4AB152517F9E516D6
:1027770035F0FA8047AB15AA16A91775F020E52E94
:10278700A4F58285F083120721FF7885E6C39FFFB2
:10279700E49400FE7C00EF252BFFEC3EFEEF252C9A
:1027A700FFEC3EFE740F2FF58274073EF583E0FDC4
:1027B700E52E75F020A429F9EA35F0FA90000D12FC
:1027C7000AAC788BE6FF18E68FF0A4FFE52B2FF510
:1027D70082E435F0F583ED120760052B02270BAF76
:1027E7002E12B2F8788B060226FD788BA630E52EDE
:1027F70075F020A4AB152517F9E51635F0FA90000A
:102807000412072130E5047884A62EE52A6488702F
:10281700158010E52EB4FF0E900712E0F520E52A8B
:10282700B4880312AF8DE52A64A86003022965788E
:1028370087E6B4010F7A007B327D01788BE6FF12C1
:10284700A20F801AE4F52BE52BC3787F96500F7AF9
:10285700007B327D01AF2B12A20F052B80E9900779
:1028670011E030E711547FFEA3E0FDEEF532EDF500
:1028770033752C03800C900711E0753200F5337522
:102887002C027410252CF582E43407F583E0FF74DD
:1028970011252CF582E43407F583E0F52F8F2EE51B
:1028A7002ED3952F4003022962E52EC378829640E6
:1028B7000302295DAB15AA16A91775F020E52EA40A
:1028C700F58285F083120721F52D7887E6B4010993
:1028D700788BE6F531F5308009E4F530787FE6143A
:1028E700F531788BA630788BE6D39531505EE4F5D9
:1028F7002BE52BC3952D504AE52E75F020A4AB157B
:102907002517F9E51635F0FA90000412072120E2A1
:102917002DE52C252B2412F582E43407F583E0FD01
:1029270090000D120AAC788BE6FF18E68FF0A4FF33
:10293700E52B2FF582E435F0F583ED120760052BC3
:1029470080AFAF2E12B2F8788B06809A788BA630BC
:0E295700E52D252CF52C052E0228A612AF8D9D
:01296500224F
:09AB330090001D12084AFFAEF06B
:10AB3C008E418F42900700E065417004A3E06542AE
:10AB4C00603A9006F0740AF0E541A3F0E542A3F0F8
:10AB5C007C007D037B017A0679F012A3BD9006F38D
:10AB6C00EFF07B017A0679F07548017D047C0012C8
:0DAB7C00A17D900700E541F0A3E542F02225
:03AC3100CCEECC9A
:10AC34009006F0741AF0A3ECF0EFA3F07C007D030F
:10AC44007B017A0679F012A3BD9006F3EFF07B0145
:10AC54007A0679F07548017D047C0012A17D7B01A0
:10AC64007A0679F07D0A7C00129A4DEF7002FF2279
:0DAC74009006F0E0647860037F00227F010D
:01AC810022B0
:10B025007A007B327D017F0112A20F74FF90070029
:10B03500F0A3F07F0A9006F0E4F0A3DFFC7B017A31
:0DB045000679F07548017D0A7C0002A17DAE
:10906A00E4F53FE53FC37882964003029194E53FD9
:10907A0075F020A4AB152517F9E51635F0FA90001E
:10908A000412072120E40302918F12AB339006F0F9
:10909A0074A1F0E53F75F020A4AB152517F9E51684
:1090AA0035F0FA90001F1207219006F1F07C007D3E
:1090BA00027B017A0679F012A3BD9006F2EFF07BEB
:1090CA00017A0679F0E4F5487D03FC12A17D7B0163
:1090DA007A0679F07D647C00129A4D8F40E540C390
:1090EA0094025002804DE5402476FF9006F0E06F2E
:1090FA006002803FAB15AA16A91775F020E53FA4B8
:10910A00F58285F083120721FFE54024FE6F600295
:10911A008021E54024FFFDE434FFFC7B017A0679D7
:10912A00F012A3BD74EF2540F582E43406F583E01E
:10913A006F6007AF3F12B025804BC2AFAB15AA16BE
:10914A00A91775F020E53FA4F58285F0831207215F
:10915A00FF7E00EEC0E0EFC0E0E53F75F020A429F5
:10916A00F9EA35F0FA90000D120AACC8E9C8CCEA5F
:10917A00CCCDEBCD7B017A0679F1D0E0FFD0E0FED1
:0A918A001206E2D2AF053F02906D1D
:0191940022B8
:02A4D5008F3FB7
:10A4D700EF75F020A4AB152517F9E51635F0FA123C
:10A4E700AB33AB15AA16A91775F020E53FA4F58283
:10A4F70085F083120721F54024819006F0F0E53FAF
:10A5070075F020A429F9EA35F0FA90001F12072107
:10A517009006F1F0AF407E0090000D120AAC78F281
:10A527007C067D011206E2E5402402FDE433FC7B54
:10A53700017A0679F012A3BD74F22540F582E4345E
:10A5470006F583EFF07B017A0679F0E5402403FDF9
:09A55700E433FCE4F54802A17DA7
:10AE0B0012B362C8ECC8C9EDC9CAEECACBEFCB907E
:10AE1B000708E0FCA3E0FDA3E0FEA3E0240AFFE4A7
:10AE2B003EFEE43DFDE43CFCD31208FD400C1290C9
:10AE3B006A12B362900708120A2C7884E6FFF4605A
:09AE4B000712A4D5788476FF22D9
:10F000007880E664F1600302F60CE4F544F5457897
:04F0100081E6601F16
:0DF01400754A0A754B1300D54BFCD54AF622
:10F021000545E5457002054464107004E544642714
:10F0310070DCC2AF7584015398FC75FFDE75FFADBE
:10F04100E4F540F53FE4F58420982EE4F544F545D8
:0EF05100209822C3E5459488E5449413501797
:0DF05F00754A0A754B1300D54BFCD54AF6D7
:10F06C000545E54570DF054480DBB28680CF859988
:10F07C003FC298E53F641A600302F14CF544F54534
:0EF08C00209822C3E5459488E544941350175C
:0DF09A00754A0A754B1300D54BFCD54AF69C
:10F0A7000545E54570DF054480DB3098928599403A
:10F0B700C298E4F544F545209822C3E5459488E5D0
:05F0C7004494135017F2
:0DF0CC00754A0A754B1300D54BFCD54AF66A
:10F0D9000545E54570DF054480DB20980302F046CD
:10F0E900859940C298E4F544F545209822C3E54541
:08F0F9009488E54494135017BC
:0DF10100754A0A754B1300D54BFCD54AF634
:10F10E000545E54570DF054480DB20980302F04697
:09F11E00859940C298D285C2997E
:0DF12700754A14754B1300D54BFCD54AF604
:06F134007599783099FD89
:0DF13A00754A0A754B1300D54BFCD54AF6FB
:10F14700C28502F5FEE53F6450600302F1DCF54439
:10F15700F545209822C3E5459488E5449413501754
:0DF16700754A0A754B1300D54BFCD54AF6CE
:10F174000545E54570DF054480DB20980302F04631
:09F18400859940C298D285C29918
:0DF18D00754A14754B1300D54BFCD54AF69E
:08F19A007599793099FDC299C5
:0DF1A200754A14754B1300D54BFCD54AF689
:08F1AF007599013099FDC29928
:0DF1B700754A14754B1300D54BFCD54AF674
:06F1C400E4F5993099FD0D
:0DF1CA00754A0A754B1300D54BFCD54AF66B
:0FF1D700C28502F5FEE53F6401703ED285C29904
:0DF1E600754A14754B1300D54BFCD54AF645
:08F1F3007599783099FDC2996D
:0DF1FB00754A14754B1300D54BFCD54AF630
:06F20800E4F5993099FDC8
:0DF20E00754A0A754B1300D54BFCD54AF626
:10F21B00C28502F5FEE53F6402600302F2E2F544AB
:10F22B00F545209822C3E5459488E544941350177F
:0DF23B00754A0A754B1300D54BFCD54AF6F9
:10F248000545E54570DF054480DB20980302F0465C
:10F25800859940C298E4F541E54013B39286E540AC
:10F2680025E0FEC3E49400EE94F0502AE5407F00C8
:10F2780025E0FEC394E0501EE54020E01FE4F5843D
:10F2880043B701758F038E468F478F828E83F05365
:10F29800B7F0F58F80037541FFE4F584D285C299F4
:0DF2A800754A14754B1300D54BFCD54AF682
:08F2B5007599783099FDC299AA
:0DF2BD00754A14754B1300D54BFCD54AF66D
:06F2CA008541993099FD19
:0DF2D000754A0A754B1300D54BFCD54AF664
:10F2DD00C28502F5FEE53F6403600302F42DF5449B
:10F2ED00F545209822C3E5459488E54494135017BD
:0DF2FD00754A0A754B1300D54BFCD54AF637
:10F30A000545E54570DF054480DB20980302F04699
:10F31A00859940C298E4F544F545209822C3E5450D
:08F32A009488E5449413501788
:0DF33200754A0A754B1300D54BFCD54AF601
:10F33F000545E54570DF054480DB20980302F04664
:10F34F00859942C298E540139286E54025E0FEC3B9
:10F35F00E49400EE94F0400302F046E5407D002572
:10F36F00E0FCC394E0400302F046E4F58443B701A8
:10F37F00758F01E54275F020A42DFFE5F03CF546B1
:10F38F008F47E4F584F543E543C394205048E4F5F3
:10F39F0044F545209822C3E5459488E544941350DD
:01F3AF001746
:0DF3B000754A0A754B1300D54BFCD54AF683
:10F3BD000545E54570DF054480DB20980302F046E6
:10F3CD000547E547AE467002054614F5828E83E586
:10F3DD0099F0C298054380B1E4F58453B7F0F58FE9
:06F3ED00F584D285C299EF
:0DF3F300754A14754B1300D54BFCD54AF636
:08F400007599783099FDC2995D
:0DF40800754A14754B1300D54BFCD54AF620
:06F41500E4F5993099FDB9
:0DF41B00754A0A754B1300D54BFCD54AF617
:10F42800C28502F5FEE53F6404600302F4DDF5449D
:10F43800F545209822C3E5459488E5449413501770
:0DF44800754A0A754B1300D54BFCD54AF6EA
:10F455000545E54570DF054480DB20980302F0464D
:10F46500859940C298E54025E0F548754900E4F5E1
:10F4750041F544F5450549E549AE4870020548148E
:10F48500F5828E83E4932541F5410545E5457002F6
:0EF4950005447004E544640270DBD285C29920
:0DF4A300754A14754B1300D54BFCD54AF685
:08F4B0007599783099FDC299AD
:0DF4B800754A14754B1300D54BFCD54AF670
:06F4C5008541993099FD1C
:0DF4CB00754A0A754B1300D54BFCD54AF667
:10F4D800C28502F5FEE53F6405600302F5F3F544D5
:10F4E800F545209822C3E5459488E54494135017C0
:0DF4F800754A0A754B1300D54BFCD54AF63A
:10F505000545E54570DF054480DB20980302F0469C
:10F51500859940C298E4F544F545209822C3E54510
:08F525009488E544941350178B
:0DF52D00754A0A754B1300D54BFCD54AF604
:10F53A000545E54570DF054480DB20980302F04667
:09F54A00859942C298D285C2994C
:0DF55300754A14754B1300D54BFCD54AF6D4
:08F5600075997F3099FDC299F5
:0DF56800754A14754B1300D54BFCD54AF6BF
:10F575007599203099FDE54025E0FCE54275F020C0
:10F58500A42400FFE5F03CF5488F49E4F541F54337
:02F59500C29919
:0DF59700754A14754B1300D54BFCD54AF690
:10F5A400854982854883E493F5993099FD0549E5B9
:10F5B40049AE487002054814F5828E83E4932541D0
:0BF5C400F5410543E543B420C8C2999F
:0DF5CF00754A14754B1300D54BFCD54AF658
:06F5DC008541993099FD04
:0DF5E200754A0A754B1300D54BFCD54AF64F
:10F5EF00C285800BE53FB40606E4F58475EF10E5A0
:0DF5FF003F6407600302F0467880F6D2AF4B
:01F60C0022DB
:1097B2007F0012B0AC20290B7A007B327D017F0042
:1097C20012A20F302C0B7A007B1E7D017F0012A2A9
:1097D2000F302817302D147A007B327D01788BE60A
:1097E200FF12A20FC228129DD9D229202B0C302D94
:1097F20009788076F1129DD9D22B302E2A302D276E
:10980200C22E12B3BAE4FDFF12B29A7BFF7AB0798C
:10981200D812B12E7D01E4FF12B29A7BFF7AB079A1
:10982200E612B12E12F000302F0B7B017A0779027B
:1098320012A5EAC22F12B362C8ECC8C9EDC9CAEEBA
:10984200CACBEFCB90070C1209BBEF245AFFE43EC0
:10985200FEE43DFDE43CFCD31208FD500F12B3625E
:1098620090070C1209D4D31208FD401212B3629071
:10987200070C120A2C7B017A0679FA129972202DB2
:109882001212B362E47B2C7A01F9F8C31208FD507C
:0498920002D22D22AF
:0EB3AC001264021297B212AE0B1258A380F573
:108F31004D656D6F727920746573742E2E2E004D00
:108F4100656D6F7279206572726F722062616E6BEE
:108F51002025626400005EBCE2613FDD83C29C7E2D
:108F610020A3FD1F419DC3217FFCA2401E5F01E3A1
:108F7100BD3E6082DC237D9FC1421CFEA0E1BF5D3E
:108F81000380DE3C62BEE0025CDF81633D7C22C087
:108F91009E1D43A1FF4618FAA427799BC584DA38A0
:108FA10066E5BB5907DB856739BAE406581947A559
:108FB100FB7826C49A653BD987045AB8E6A7F91B02
:108FC10045C6987A24F8A6441A99C7257B3A64863F
:108FD100D85B05E7B98CD2306EEDB3510F4E10F26C
:108FE100AC2F7193CD114FADF3702ECC92D38D6F09
:108FF10031B2EC0E50AFF1134DCE90722C6D33D1D6
:109001008F0C52B0EE326C8ED0530DEFB1F0AE4CEE
:109011001291CF2D73CA947628ABF517490856B42F
:10902100EA6937D58B5709EBB536688AD495CB29D0
:1090310077F4AA4816E9B7550B88D6346A2B759789
:10904100C94A14F6A8742AC896154BA9F7B6E80AB6
:1090510054D7896B35000000002B6096CBDDEE0004
:099061002C96CBDDE5EEF7FAFDDB
:05ADD800C1B2017B0A7D
:10B34F0074FFF571F570F56FF56EAF71AE70AD6F8F
:02B35F00AC6ED2
:01B3610022C9
:10A3BD0015791579A879ECF608EDF6157915791555
:10A3CD0079A879C6EBC608C6EAC608C6E9C6E57916
:04A3DD0024FCF579EE
:10A3E100F80808E4F6A879F608F6E5792407F9A84B
:10A3F10079E6FE08E6FFC3099719E76480F8EE6481
:10A4010080985037E5792404F8CBE6CB08E6FA08C2
:10A41100E6F98F828E83120721A879080866FFE585
:10A42100792403F8EFF6E6908F5693A8790808F699
:10A43100A8790806E61870B20680AFA8790808E680
:01A44100FF1B
:07A44200E5792409F57922F8
:0BB3D400ED6F78A7F6E6908F5693FF10
:01B3DF00224B
:0300A30002AB8924
:10AB8900C0E0C083C082C0D0E8C0E0EEC0E0EFC042
:10AB9900E0E59830E1055398FDD232E59830E0249C
:10ABA900787AE62401FFE433FEEF64404E700280B8
:10ABB90010787AE60624F0F582E43408F583E599FD
:10ABC900F05398FED0E0FFD0E0FED0E0F8D0D0D02E
:06ABD90082D083D0E032BF
:0AA17D008B438A4489458C468D47C8
:10A18700E4787AF6758401D284E54824FF929BE44B
:10A1970078A8F678A8E6C39547E5466480F8748002
:05A1A700985060C23277
:0DA1AC00754914754A1300D54AFCD549F6D3
:10A1B900E54724FFFFE54634FFFE78A8E66F700106
:10A1C900EE701EC2ACAB430545E545AA44700205D5
:10A1D9004414F9120708F5993032FDC284D2AC80D3
:10A1E90016AB430545E545AA447002054414F91226
:10A1F9000708F5993032FD7F0112B0AC78A80680C6
:05A2090090C284AF4784
:01A20E00222D
:0A9A4D008B418A4289438C448D4509
:109A570012B36278A9120A20E478A8F612B362EC6E
:109A6700C0E0EDC0E0EEC0E0EFC0E078A91209AFBA
:109A7700CBEFCBCAEECAC9EDC9C8ECC8D0E0FFD05E
:109A8700E0FED0E0FDD0E0FCC3EF9BFFEE9AFEEDD9
:109A970099FDEC98FCE47B01FAF9F8C31208FD5034
:109AA700037F0022787AE6FED3940040539008F0B3
:109AB700E0FDB478037F0122ED54F8647860037FFA
:109AC70000229008F0E05407240278A8F66E703060
:109AD700787AE6D39545E5446480F8748098400623
:109AE700AE44AF458006787AE6FF7E00A843AC42D5
:109AF700AD417B017A0879F01206E278A8E6FF22E9
:089B07007F0112B0AC029A6369
:07B3E000E4787AF6D2322274
:10AC8200EF7025F5847598D0F584759115F5847566
:10AC9200C90875CBFFED90905593F5CA75C804E4C9
:10ACA200F584D2ACC2BC80267584017598D0E4F5D7
:10ACB20084E589540F4420F589758E02ED90905FEA
:10ACC20093F58DD28E43E74043F74012B3E0D2AF03
:01ACD200225F
:10A82400900930120A5100000000900934120A51B4
:10A83400000000009008E77464F0E478A8F678A8B3
:10A84400E6FFC394025043EF25E025E024E8F582B7
:10A85400E43408F583E4F0EF25E025E024E9F5820B
:10A86400E43408F583E4F0EF25E025E024EAF582FA
:10A87400E43408F583E4F0EF25E025E024EBF582E9
:0AA88400E43408F583E4F00680B424
:01A88E0022A7
:10B1C900D2AFD2A9C2BBE4F584E589540F4401F595
:0FB1D90089758E02758CAFE4F58AD28C02A8249A
:0295D800157903
:1095DA00A879E4F6A879E6FFC3940240030296C785
:1095EA00EF25E025E024EBF582E43408F583E0FF7B
:1095FA00D39400500302969CE625E025E024E9F581
:10960A0082E43408F583E0600302969CEF30E019A7
:10961A00E6FF25E025E024EBF582E43408F583E053
:10962A00D3940140047D0080067D01A879E6FF12EB
:10963A00A748A879E6FF25E025E024EBF582E43483
:10964A0008F583E0B401057D0112A748A879E6FF71
:10965A0025E025E024EBF582E43408F583E014F0F4
:10966A00EF25E025E024EBF582E43408F583E06099
:10967A0021E6FF25E025E024EAF582E43408F583B3
:10968A00E0FEEF25E025E024E9F582E43408F583DD
:10969A00EEF0A879E6FF25E025E024E9F582E43436
:1096AA0008F583E06011EF25E025E024E9F582E47E
:0D96BA003408F583E014F0A879060295DE6F
:0396C70005792200
:03000B0002A05000
:10A05000C0E0C0F0C083C082C0D0E8C0E0E9C0E08A
:10A06000EAC0E0EBC0E0ECC0E0EDC0E0EEC0E0EF45
:10A07000C0E0758CAF900930E0FCA3E0FDA3E0FEEA
:10A08000A3E02401FFE43EFEE43DFDE43CFC900936
:10A0900030120A2C9008E7E014F0E07025900934A3
:10A0A000E0FCA3E0FDA3E0FEA3E02401FFE43EFE0C
:10A0B000E43DFDE43CFC900934120A2C9008E7745E
:10A0C00064F01295D812B1A7D0E0FFD0E0FED0E046
:10A0D000FDD0E0FCD0E0FBD0E0FAD0E0F9D0E0F831
:0BA0E000D0D0D082D083D0F0D0E0328E
:10B052001579A879EDF61579A879EFF6A879E6FFC2
:10B06200C39402501308E6FEEF25E025E024E8F53C
:0DB0720082E43408F583EEF00579057922BB
:10A20F0015791579A879EAF608EBF61579A879ED9D
:10A21F00F61579A879EFF6A879E6FFC39402506A8C
:10A22F00EF25E025E024EBF582E43408F583E070B8
:10A23F0059E6FB25E025E024E9F582E43408F583AF
:10A24F00E0704708E625E004FFA879E6FA25E02547
:10A25F00E024EBF582E43408F583EFF00808E6FE1E
:10A26F0008E6FF7C007D0A1207E9EA25E025E024D5
:10A27F00EAF582E43408F583EFF0EB25E025E024DE
:10A28F00E9F582E43408F583E4F0E5792404F579FF
:01A29F00229C
:0EA748001579A879EDF61579A879EFF615794F
:10A75600A87908E6FFC394025024EF25E025E024FB
:10A76600E8F582E43408F583E06013A8790808E682
:10A7760070047F0180027F00A8790808EFF6A879A7
:10A78600A68475840FA87908E6FF700BA8790808D7
:10A79600E624FF9286800DEFB40109A8790808E641
:09A7A60024FF9287A879E6F584EE
:07A7AF000579057905792207
:10B36200C2AF900930E0FCA3E0FDA3E0FEA3E0FF42
:02B37200D2AF58
:01B3740022B6
:10B37500C2AF900934E0FCA3E0FDA3E0FEA3E0FF2B
:02B38500D2AF45
:01B3870022A3
:10B0AC001579A879EFF6A879E67005787CF608F69C
:10B0BC00303016787BE675F064A4FFC3787DE69F8C
:0CB0CC0018E695F0500375FFA5057922E9
:10B1E800D230E4787CF608F6EF787B6003F68002CC
:0FB1F800760A75FF0775FFA5E4F58475EF04224D
:10B38800C230E4787CF608F6787B76FF75FFDE75C8
:03B39800FFAD22E4
:10B1A700787D06E618700106303016787BE675F074
:10B1B70064A4FFC3787DE69F18E695F0500375FFFA
:02B1C700A522BF
:04B103008E448F45A2
:10B10700E4F546F547C3E5479545E54695445016AA
:10B117007FE87E0312A90D7F0112B0AC0547E54712
:06B1270070E3054680DF25
:01B12D0022FF
:10A8FA0043A0F075840F43A60FC290C294D2957FED
:03A90A00017E00CB
:04A90D008E648F6560
:10A91100D3E56594FAE5649400500EEFD3940040BA
:10A92100407E1600DEFD1F80F2856466856567D373
:10A93100E56794FAE566940040157FFA7E0012A956
:10A941000D74062567F56774FF3566F56680E0D3FB
:10A95100E5659400E56494004007AF67AE6612A90F
:01A961000DE8
:01A9620022D2
:10A9630075500075510075524A7B007A0079487D15
:01A9730002E1
:08A974008B4C8A4D894E8D4F7A
:10A97C007F0112B0ACAB50AA51A95212081F24008F
:10A98C00FFE5F034E0FE854C53854D54854E55E47F
:10A99C00FDEDC3954F501BEF2DF582E43EF583E49E
:10A9AC0093AB53AA54A9558D827583001207600D81
:0FA9BC0080DFAB50AA51A952E4854FF002088208
:109BD000754112754234754900754A00754B437BD7
:079BE000007A0079417D02CB
:089BE7008B458A4689478D4831
:109BEF007880E664F16003029C8412B388C2AFE40C
:109BFF00F58443B701758F01AB49AA4AA94B1208E7
:109C0F001F2400FFE5F034E078A8F608EFF6AA4627
:109C1F00A94778ACA64508C6EAC608C6E9C6E478DF
:109C2F00AAF678AAE6C39548503278ACCBE6CB08B3
:109C3F000806E618CAE6CA70010614F91207087872
:109C4F00ABF6E6FF78A80806E618CCE6CC7001065E
:109C5F0014F5828C83EFF078AA0680C6E4F58F5353
:109C6F00B7F0AB49AA4AA94B8548F0120882D2AF88
:059C7F00E4FF12B1E852
:019C840022BD
:10AD71007880E664F17046C2AF12B388E4F584438B
:10AD8100B701758F0378A976E008F678A8F678A957
:10AD9100E6FE08E6F5828E83E4F07F0112B0AC781E
:10ADA100AAE426F618740236F61806E6C39408409B
:0DADB100DDE4F58F53B7F0D2AFFF12B1E82B
:01ADBE002272
:109DD90012AD71E4F543F544F549754A00754B43F5
:109DE900FB7A00798D7D16129BE7129BD0E4F54032
:109DF900E540C3787F965073E4F53FAB15AA16A9E1
:109E09001775F020E53FA4F58285F08312072160DC
:109E190056E53F75F020A429F9EA35F0FA90000DCE
:109E2900120AAC788AE68540F0A429F9EA35F0FAF5
:109E3900EBC0E0EAC0E0E9C0E0AB15AA16A91775C6
:109E4900F020E53FA4F58285F083120721FD7549CD
:109E590000754A00754B43D0E0F9D0E0FAD0E0FB39
:109E6900129BE7053F809405408085129BD0E478DA
:029E790080F671
:019E7B0022C4
:0296CA008F44CB
:1096CC00E4F54AF54BF547F55075510075524AFBD8
:1096DC007A00798D7D1612A97412A963E549643458
:1096EC007004E54864127003434701E4F546E5460F
:1096FC00C3787F96400302979DE4F545AB15AA16F7
:10970C00A91775F020E545A4F58285F08312072191
:10971C00607AE5446054E54575F020A429F9EA35F2
:10972C00F0FA90000D120AAC788AE68546F0A4296E
:10973C00F9EA35F0FAEBC0E0EAC0E0E9C0E0AB15BD
:10974C00AA16A91775F020E545A4F58285F08312B9
:10975C000721FD75500075510075524AD0E0F9D0C3
:10976C00E0FAD0E0FB12A974801DAB15AA16A9175C
:10977C0075F020E545A4F58285F083120721254B71
:10978C00F54BE4354AF54A0545029708054602961D
:10979C00FA12A963E54964347004E5486412700355
:0597AC00434702AF4736
:0197B1002295
:02A7B6008F62B0
:10A7B80030316812A8FAD296E4F5637F0A7E001257
:10A7C800A90D30A7090563E563C394C840EDC29697
:10A7D80012A909C295D29075840F75A6FF12A9090E
:10A7E800E56254F0FFE5A054014FF5A0A21E929433
:10A7F80012A909D29612A909C29612A909E562C43A
:10A8080054F0FFE5A054014FF5A0A21E929412A99E
:0BA8180009D29612A909C29612A909E4
:01A823002212
:10AFF5008F4453A00FE54454F042A0D29612A909FC
:10B00500C29612A90953A00FE544C454F042A0D238
:10B015009612A909C29612A9097F647E0002A90D9C
:10A6D400E478A8F608F6C296C295C29475840F75FC
:10A6E400A6FF43A503D290D29153A00143A020D248
:10A6F400967F01FE12A90DC2967F017E0012B1035E
:10A704007F2012AFF512A8FAD2967F647E0012A9B8
:10A714000D30A703C23122D231C21E7F2412A7B644
:10A72400C21E7F0B12A7B6C21E7F2012A7B6C21E7E
:10A734007F0C12A7B6C21E7F0112A7B6C21E7F06E7
:03A7440012A7B6A3
:01A7470022EF
:0DB3BA00C21E7F0112A7B6E4FDFF02B29A89
:10B39B00EF6006C21E7F0F8004C21E7F0C12A7B681
:01B3AB00227F
:06B2940078A8E6FF7D032F
:10B29A00ED5403C43354E0FEEF541F44804EFFC202
:04B2AA001E02A7B623
:10B326008F61E561640D600BE561640A6005D21EFC
:06B3360012A7B6AF612270
:10B180008B728A738974AB72AA73A97412070860F0
:10B19000150574E5747002057314F9120708FFD2DF
:07B1A0001E12A7B680E02299
:10B22500EF540778AAF6EF30E306E64420F68004EB
:0CB2350078AAE6F678AAE644C0F6F5C850
:01B2410022EA
:0285BF008F44E7
:1085C10012B3BA7D017F0212B29A7BFF7A8F7931A1
:1085D100125496E478A9F612B388C2AFE478A8F6EB
:1085E10078A8E6FFC39544400302870412B225121E
:1085F100B2947FDA12B326902000AF82AE83C3EF2C
:1086010094FFEE94FF5005E4F0A380EE902000AFBC
:1086110082AE83C3EF94FFEE94FF500CE0600678C6
:10862100A976018003A380E778A9E66003028704A5
:1086310012B2947FD912B326902000AF82AE83C3C9
:10864100EF94FFEE94FF50067455F0A380ED902057
:1086510000AF82AE83C3EF94FFEE94FF500EE0644F
:1086610055600678A976018003A380E578A9E660C4
:108671000302870412B2947FD812B326902000AF70
:1086810082AE83C3EF94FFEE94FF500674AAF0A369
:1086910080ED902000AF82AE83C3EF94FFEE94FF94
:1086A100500EE064AA600678A976018003A380E5F4
:1086B10078A9E6704E12B2947FD712B326902000AB
:1086C100AF82AE83C3EF94FFEE94FF500674FFF0C8
:1086D100A380ED902000AF82AE83C3EF94FFEE94B0
:1086E100FF500DE0F4600678A976018003A380E6CF
:1086F10078A9E6700E12B2947FD612B32678A80636
:108701000285E1D2AFE4FF12B1E812B22578A9E601
:10871100601A7D0212B29A7BFF7A8F794078A8E6BF
:0C872100F5481254967F0012B0AC80F9AD
:01872D002229
:10A88F00E4F58475A338F5A275A10475840F759C42
:10A89F00FF759DFF759EFF759FFF75F8FF75E8FFAC
:10A8AF0075D8FF75C8FFFF12B225902000E078A879
:10A8BF00F67455F0E064556008E6F0E4F584F5A30E
:10A8CF002278A8E6F07F0812B225E078A8F674AADD
:10A8DF00F0E0B4AA0AE6F0E4FF12B2257F10227866
:0AA8EF00A8E6F0E4FF12B2257F088E
:01A8F900223C
:10383400506C6561736520696E73657274206D6F79
:1038440064756C65002020202741443539302720D9
:103854002830783734292020202000202020206997
:103864006E746F20706F727420302020202020002E
:10387400202755696E202B2D31305627202830788B
:1038840036312920002020202020696E746F20709A
:103894006F72742031202020200020202020274413
:1038A4006F75742720283078343029202020002098
:1038B40020202020696E746F20706F727420352070
:1038C400202020002020202752656C616973272066
:1038D4002830783431292020002020202020696ECF
:1038E400746F20706F7274203620202020002020F6
:1038F40020274F7074496E272028307832312920D0
:103904002020002020202020696E746F20706F72A8
:10391400742037202020200020002A2A2000202A7A
:103924002A00202020416464726573733A202025A4
:103934003034580020205265766973696F6E3A20DE
:103944002025730057726F6E672043504C442066E5
:1039540069726D7761726500536C6176652061648C
:1039640064723A20256264005265713A202530322F
:10397400626420213D204163743A20253032626420
:10398400004F76657263757272656E74203E312ED7
:103994003541206F6E00202020323456206F75741C
:1039A4007075742021212120202000202020536CB8
:1039B40061766520616464723A2025626400524530
:1039C400534554004F76657263757272656E742048
:1039D4003E302E3541206F6E0020202020355620A9
:1039E4006F757470757420212121002020202053CC
:1039F4006C61766520616464723A202562640020FB
:103A040020202055203D2025312E3266205600549A
:103A1400303A2025312E326620430054313A202595
:103A2400312E32662043004F666620696E202531B0
:103A34002E316620732020004F6E20696E202531C0
:103A44002E31662073202020004F6E20202020205D
:103A5400202020202020004F6666202020202020C7
:103A6400202020200056415253005343532D32301E
:103A740030312D415050002449643A207363735F00
:103A8400323030305F6170702E632032383734202A
:103A9400323030352D31312D31352030383A34370C
:103AA4003A31345A207269747420240004080000E6
:103AB40001543000000000000001089402000000DE
:103AC40000000000000000000000000004080000E6
:103AD40001543100000000000001089802000000B9
:103AE40000000000000000000000000004080000C6
:103AF40001543200000000000001089C0200000094
:103B040000000000000000000000000004080000A5
:103B14000154330000000000000108A0020000006E
:103B24000000000000000000000000000408000085
:103B34000154340000000000000108A40200000049
:103B44000000000000000000000000000408000065
:103B54000154350000000000000108A80200000024
:103B64000000000000000000000000000408000045
:103B74000154360000000000000108AC02000000FF
:103B84000000000000000000000000000408000025
:103B94000154370000000000000108B002000000DA
:103BA40000000000000000000000000004180000F5
:103BB4000141444330300000000108B40400000017
:103BC40000000000000000000000000004180000D5
:103BD4000141444330310000000108B804000000F2
:103BE40000000000000000000000000004180000B5
:103BF4000141444330320000000108BC04000000CD
:103C04000000000000000000000000000418000094
:103C14000141444330330000000108C004000000A7
:103C24000000000000000000000000000418000074
:103C34000141444330340000000108C40400000082
:103C44000000000000000000000000000418000054
:103C54000141444330350000000108C8040000005D
:103C64000000000000000000000000000418000034
:103C74000141444330360000000108CC0400000038
:103C84000000000000000000000000000418000014
:103C94000141444330370000000108D00400000013
:103CA40000000000000000000000000001320000DD
:103CB40000446F7574300000000108D80000000053
:103CC400003F8000003F800000000000013200003F
:103CD40000446F7574310000000108D90000000031
:103CE400003F8000003F800000000000013200001F
:103CF40000446F7574320000000108DA000000000F
:103D0400003F8000003F80000000000001320000FE
:103D140000446F7574330000000108DB00000000EC
:103D2400003F8000003F80000000000001320000DE
:103D340000446F7574340000000108DC00000000CA
:103D4400003F8000003F80000000000001320000BE
:103D540000446F7574350000000108DD00000000A8
:103D6400003F8000003F800000000000013200009E
:103D740000446F7574360000000108DE0000000086
:103D8400003F8000003F800000000000013200007E
:103D940000446F7574370000000108DF0000000064
:103DA400003F8000003F800000000000013200005E
:103DB4000052656C30000000000108D400000000CF
:103DC400003F8000003F800000000000013200003E
:103DD4000052656C31000000000108D500000000AD
:103DE400003F8000003F800000000000013200001E
:103DF4000052656C32000000000108D6000000008B
:103E0400003F8000003F80000000000001320000FD
:103E14000052656C33000000000108D70000000068
:103E2400003F8000003F80000000000001320000DD
:103E34000044696E30000000000108E0000000004A
:103E4400000000000000000000000000013200003B
:103E54000044696E31000000000108E10000000028
:103E6400000000000000000000000000013200001B
:103E74000044696E32000000000108E20000000006
:103E840000000000000000000000000001320000FB
:103E94000044696E33000000000108E300000000E4
:103EA4000000000000000000000000000203000009
:103EB40000506572696F6400000108E400000000AE
:103EC40000456100003F8000000000000000000089
:103ED40000000000000000000000000000000000DE
:0C3EE400000000000000000000000000D2
:10ADDD00017F010315FF3AB0C111C10CC112C1139E
:10ADED00C10DC10EC10FC110010C000411000000F6
:0DADFD0000040D000000000408000000002C
:107A3F0075840F75A4F575A5FF75A6FF75A70FE4DF
:107A4F00F584F5BA75BC9875E880F5D1F58475D1D4
:107A5F0003F58475D48075840175D480FDFF12B24F
:107A6F009A7B74E4FDFF12AF56EF70297BFF7A38D3
:107A7F0079341254967BFF7A3879491254967BFFEA
:107A8F007A38795F125496E4FF12AADCEF7006FF82
:107A9F0012B0AC80F27B617D01E4FF12AF56EF7044
:107AAF00297BFF7A3879341254967BFF7A387974B0
:107ABF001254967BFF7A387989125496E4FF12AAF2
:107ACF00DCEF7006FF12B0AC80F27B407D05E4FF67
:107ADF0012AF56EF70297BFF7A3879341254967BA8
:107AEF00FF7A38799E1254967BFF7A3879B3125405
:107AFF0096E4FF12AADCEF7006FF12B0AC80F27BA7
:107B0F00417D06E4FF12AF56EF70297BFF7A38797B
:107B1F00341254967BFF7A3879C81254967BFF7AC9
:107B2F003879DD125496E4FF12AADCEF7006FF12CB
:107B3F00B0AC80F27B217D07E4FF12AF56EF7029C6
:107B4F007BFF7A3879341254967BFF7A3879F212A8
:107B5F0054967BFF7A397907125496E4FF12AADC08
:107B6F00EF7006FF12B0AC80F212A82415791579C8
:107B7F001579A87976000876000876001579A87926
:107B8F00E4F61579A879F6FB7D017F74126D38152F
:107B9F007915791579A87976000876000876001599
:107BAF0079A879E4F61579A8797601FB7D017F61D3
:107BBF00125CA2157915791579A8797600087600E7
:107BCF000876001579A879E4F61579A8797605FB7A
:107BDF007D017F4012844B157915791579A8797637
:107BEF00000876000876001579A879E4F61579A8CB
:107BFF00797606FB7D017F4112844B157915791536
:107C0F0079A87976000876000876001579A879E4C6
:0F7C1F00F61579A8797607FB7D017F210293C0C6
:028143008F4467
:108145007D017F0012B0527D007F0112B052E49094
:108155000988F0900988E0FFC39403500B129B0F28
:10816500900988E004F080EB120003E544604DE4DB
:10817500900988F0900988E0FFC39404501474D4E2
:108185002FF582E43408F583E4F0900988E004F0E3
:1081950080E2E4900988F0900988E0FFC3940850D4
:1081A5001474D82FF582E43408F583E4F090098837
:1081B500E004F080E2E49008E4F0A3F0E49009889C
:1081C500F0900988E0FFC39408500FEF2408FF12D0
:1081D500B2F8900988E004F080E7E4FDFF12B29A56
:1081E500E4900988F07B007A00799312000E7C00F8
:1081F5007D021207E9C374079FFFE49EFE9009887C
:10820500E0C39FEE6480F874809850117BFF7A3943
:10821500791C12B12E900988E004F080C87BFF7AA2
:1082250039791E12B12E7B007A00799312B12E7B1B
:10823500FF7A39792212B12E7D01E4FF12B29A7BC1
:10824500FF7A397926788DE6F54808E6F54912541E
:10825500967D02E4FF12B29A900988740AF07BFFBA
:108265007A3A797B12000E900988E0FDC39FEE648F
:1082750080F87480985011ED903A7B9364206008E3
:10828500900988E004F080D6900988E0247CF9E420
:10829500343A7548FFF549894A754B00754C067B9C
:1082A500017A09798912ABDF7B017A0979897D2009
:1082B50012B242E412074E754801754909754A899B
:0982C5007BFF7A397938025496E6
:10AADC00E4F58420110FD211F58475D103F5BA7504
:0DAAEC00BC9875E880C374079F5407F5BB44
:0DAAF90075440275451300D545FCD544F6A3
:10AB0600C2AFC2EDD2EC30EDFDD2AFAFBFEFFFADBD
:10AB1600BEED9009A3CFF0A3EFF0C3E094E890094F
:0CAB2600A3E0940350047F0180027F0034
:01AB32002200
:106FF900E490099CF012B362C8ECC8C9EDC9CAEEA5
:10700900CACBEFCB900850E0FCA3E0FDA3E0FEA3C0
:10701900E0240AFFE43EFEE43DFDE43CFCD3120813
:10702900FD501A12B362900850E0F8A3E0F9A3E00A
:10703900FAA3E0FBD31208FD500302729712B36260
:10704900900850120A2CE490099DF090099DE0FFE8
:10705900C3940140030272A67B017A09799B12A0AD
:10706900EB90099BE0C4540F640260617A007B6471
:107079007D017F0112A20F20134B12B3BAE4FDFF69
:1070890012B29A7BFF7A39794812B12E7D01E4FF59
:1070990012B29A90099DE0FFD39400400B7BFF7ACE
:1070A90039795C8F481254967D02E4FF12B29A7BBB
:1070B900FF7A39796C75480290099BE0FFC4540F37
:1070C900F549125496D21390099C7401F090099DC8
:1070D900E0FF75420175430975449E754503E4FB5C
:1070E9007D01128DF690099EE020E3030271797A01
:1070F900007B647D017F0112A20F20124E12B3BAE8
:10710900E4FDFF12B29A7BFF7A3979851254967D94
:1071190001E4FF12B29A7BFF7A39799A1254967D6B
:1071290002E4FF12B29A90099DE0FFD39400400B4C
:107139007BFF7A3979AF8F481254967D037F0F12FE
:10714900B29A7BFF7A3979C2125496D2127F03120E
:10715900AADCEF601590099DE0FF12B207C2127F09
:107169000312AADCEF70F812B3BA90099C7401F00B
:1071790012B362E47B64FAF9F8C31208FD40030212
:10718900728E90099DE0FF7542017543097544A10E
:107199007545027B037D02128DF69009A1E0C4F8C2
:1071A90054F0C868FCA3E0C4540F48FDE41203B6C8
:1071B900E4FBFA79C8784012019EE4FBFA798078F9
:1071C900451202A7E4FBFA79907840120344600261
:1071D900500302727A200C4912B3BA7A007B647D9B
:1071E900017F0112A20FE4FDFF12B29A7BFF7A39E7
:1071F90079C81254967D01E4FF12B29A7BFF7A395D
:1072090079DD1254967D02E4FF12B29A90099DE04D
:10721900FFD39400400B7BFF7A3979EF8F481254E2
:10722900967D03E4FF12B29A9009A1E0C4F854F0E4
:10723900C868FCA3E0C4540F48FDE41203B6E4FB9C
:10724900FA79C8784012019EE4FBFA7980784512F0
:1072590002A78F4B8E4A8D498C487BFF7A3A790376
:10726900125496D20C9008E67401F090099CF080B3
:1072790014300C1190099DE0FF9008E6E06F70054D
:10728900C20C12B3BA90099DE004F00270542012A6
:1072990006200C0330130690099C7401F090099C98
:0272A900E0FF04
:0172AB0022C0
:10B2F8001579A879EFF6A879E62454F582E434089C
:08B30800F5837401F0057922C0
:05B3EC008F397F0022F3
:10B07F008B398A3A893B120708AB3CAA3DA93E128D
:10B08F00074EAB39AA3AA93B900001120721AB3CFE
:0DB09F00AA3DA93E9000011207607F022229
:10872E0030140312B3BAE4FDFF12B29A7BFF7A3A09
:10873E007913900894E0FCA3E0FDA3E0FEA3E0F51E
:10874E004B8E4A8D498C481254967D01E4FF12B22D
:10875E009A7BFF7A3A791F900898E0FCA3E0FDA37C
:10876E00E0FEA3E0F54B8E4A8D498C481254967D5F
:10877E0002E4FF12B29AD39008E5E094009008E468
:10878E00E0940050030288559008D8E070030288E8
:10879E0055E50C605912B362C3EF9514FFEE9513B5
:1087AE00FEED9512FDEC9511FCE41203B1E4FBFA1B
:1087BE0079C878421202A7ECC0E0EDC0E0EEC0E04E
:1087CE00EFC0E09008E4E0FCA3E0FDE41203B6D0B5
:1087DE00E0FBD0E0FAD0E0F9D0E0F81200A98F4B20
:1087EE008E4A8D498C487BFF7A3A792B806B12B377
:1087FE0062C3EF9514FFEE9513FEED9512FDEC9509
:10880E0011FCE41203B1E4FBFA79C878421202A714
:10881E00ECC0E0EDC0E0EEC0E0EFC0E09008E4E0B8
:10882E00FCA3E0FDE41203B6D0E0FBD0E0FAD0E00A
:10883E00F9D0E0F81200A98F4B8E4A8D498C487BF7
:10884E00FF7A3A793C80129008D8E07BFF60067A76
:10885E003A794D80047A3A795B1254967D03E4FF9F
:10886E0012B29A7BFF7A3A79691254962014092033
:10887E000806300D037F0122A208920DA209920E66
:0B888E00A20A920FA20B92107F0022A2
:10B2790035F0FA7B0190098AE0FCA3E0FDA3E0FE2A
:03B28900A3E0FF40
:08B28C00C2AF120971D2AF221A
:1058A30012B362AB0BAA0AA909A808C31208FD40E8
:1058B30003025CA112B3628F0B8E0A8D098C0890D0
:1058C30008E4E07002A3E0702E900864E06028E42E
:1058D300F0157915791579A879760108760808768F
:1058E300D81579A879F61579A8797605FB7D027F15
:1058F3004012844B025A35D39008E5E09400900897
:10590300E4E094005003025A35900864E0603DE4FB
:10591300F09008D8E0F50C157915791579A8797602
:10592300010876080876D81579A879E4F61579A8D8
:10593300797605FB7D027F4012844B9008D8E0A363
:10594300F012B3628F148E138D128C119008D8E06D
:105953007003025A3512B362ECC0E0EDC0E0EEC052
:10596300E0EFC0E09008E4E0FEA3E0FF7C007D648C
:10597300120B02EF2514FBEE3513FAED3512F9EC99
:105983003511F8D0E0FFD0E0FED0E0FDD0E0FCD34D
:105993001208FD4003025A35E50C70047F018002B2
:1059A3007F008F0C157915791579A879760008761B
:1059B3000008760C1579A879E4F61579A8797605A7
:1059C300FB7D027F4012844B9008D9E50CF09009CF
:1059D300887401F0E50C701F157915791579A8798C
:1059E30076010876090876881579A87976011579FC
:1059F300A8797605FB801E157915791579A879762E
:105A0300010876090876881579A87976021579A8A8
:105A13007976057B007D027F4012844B12B3628F3F
:105A2300148E138D128C1112B3628F108E0F8D0E84
:105A33008C0DE4FFFEFDFCAB10AA0FA90EA80DD33D
:105A43001208FD407C12B362C8ECC8C9EDC9CAEEA6
:105A5300CACBEFCBE5102464FFE4350FFEE4350E2B
:105A6300FDE4350DFCC31208FD4056E4F510F50FB7
:105A7300F50EF50D900988F0157915791579A87942
:105A830076010876090876881579A879760115795B
:105A9300A8797605FB7D027F4012844B1579157931
:105AA3001579A87976010876090876881579A87991
:105AB30076021579A87976057B007D027F401284F2
:105AC3004BE4900988F0900988E0FFC3940850469E
:105AD300157915791579A879760108760908768AF2
:105AE3001579A879EFF61579A879E4F6FB7D037F9C
:105AF30074126D38900989EFF0D394004010900927
:105B030088E075F004A42494F9740812B27990091A
:105B130088E004F080B0E4900988F0900988E0FF01
:105B2300C394085047157915791579A87976010832
:105B3300760908768A1579A879EFF61579A8797622
:105B4300017B007D037F60125CA2900989EFF0D393
:105B530094004010900988E075F004A424B4F9740B
:105B63000812B279900988E004F080AF9009887434
:105B730011F0900988E0FFC39418505274542FF524
:105B830082E43408F583E0603D900988E02454F50D
:105B930082E43408F583E4F074C82FF9E43408157B
:105BA3007915791579A879760108F608C6E9C6EF5B
:105BB30024F01579A879F61579A87976057B007D07
:105BC300027F4012844B900988E004F080A490097E
:105BD300887418F0900988E0FFC3941D50527454E0
:105BE3002FF582E43408F583E0603D900988E024D2
:105BF30054F582E43408F583E4F074BC2FF9E434FB
:105C030008157915791579A879760108F608C6E992
:105C1300C6EF24E81579A879F61579A87976067B75
:105C2300007D027F4112844B900988E004F080A438
:105C3300E4900988F0900988E0FFC3940450347419
:105C4300E02FF9E43408157915791579A8797601E7
:105C530008F608C6E9C61579A879EFF61579A87983
:105C630076077B007D037F211293C0900988E004AF
:105C7300F080C2E4FF12AADCEF24FF92087F011236
:105C8300AADCEF24FF92097F0212AADCEF24FF9221
:0E5C93000A7F0312AADCEF24FF920B120BE62D
:015CA10022E0
:1000A60002045BE86480F8E933E83360110460F029
:1000B600ED33EC337009E8FCE9FDEAFEEBFF2204C0
:1000C60060DED3EB9FEA9EE99DE8C2E78CF0C2F7BB
:1000D60095F0400CE8CCF8E9CDF9EACEFAEBCFFB87
:1000E60012042685D0F05804700320D5B3E80470B6
:1000F600075002B2D502046592D5EC0460F7E4CC51
:10010600C0E0C398F8603B94186008400DD0E0FB4F
:1001160002043DE4FBFAC9FC8028E830E406E4C9A1
:10012600FBE4CAFCE830E305E4C9CACBFCE85407A3
:100136006010F8C3E913F9EA13FAEB13FBEC13FCAE
:10014600D8F130F52FC3E49CFCEF9BFFEE9AFEED51
:1001560099FDD0E0FBEF4E4D4C701222DB030204FA
:1001660062EC2CFCEF33FFEE33FEED33FDED30E7B2
:10017600EB02043DEF2BFFEE3AFEED39FDD0E0FB3E
:1001860050130BBB0003020465ED13FDEE13FEEFE7
:0801960013FFEC13FC02043D11
:10019E00EC4D6011E8497017ED33EC3304600DE45B
:1001AE00FCFFFEFD22E933E8330470F802045B1213
:1001BE00042658046009E4CC248150062850090214
:1001CE000465284003020462C0E0EB4A7044B98023
:1001DE0006D0E0FB020451EF4E701CBD8008EBFF11
:1001EE00EAFEE9FD80EBE98DF0A4FEE5F002028760
:1001FE00E9CDF9EAFEEBFFEF89F0A4FCE5F0CE893C
:10020E00F0A42EFFE435F0CD89F0A42DFEE435F0F8
:10021E008067EF4E7005BD80D780C3EF8BF0A4AC26
:10022E00F0EE8BF0A42CFCE435F0F8EF8AF0A42C61
:10023E00E5F038FCE433CB8DF0A42CFCE5F03BF874
:10024E00EE8AF0A42CFCE5F038F8E433CF89F0A464
:10025E002CFCE5F038CF3400CE89F0A42FFFE5F06A
:10026E003EFEE433C98DF0A42EFEE5F039CD8AF0C2
:10027E00A42FFFE5F03EFEE43DFD33D0E0FB50073A
:10028E000BBB000F020465EC2CFCEF33FFEE33FECC
:06029E00ED33FD02043DFA
:1002A400020465EC5D046005E85904700302045B14
:1002B400120426580460F6EC4860F2EC7004FDFE6B
:1002C400FF22C860DB2481C85009C398600250062D
:1002D4000204629850CAF582E9294B4A7005AB8240
:1002E40002045175F0007C1A7880C3EF9BEE9AEDFE
:1002F40099400DC3EF9BFFEE9AFEED99FDE842F0A5
:10030400DC23ACF0D0E0FFD0E0FED0E0FDAB8220F7
:10031400E7101BEB60BAEC2CFCEF33FFEE33FEED81
:1003240033FD02043DE803F830E705C0F075F00042
:10033400EF2FFFEE33FEED33FD40B830E7C280AA65
:1003440074F8CC6480CCC86480C8F582046043C36C
:10035400EB9FF5F0EA9E42F0E99D42F0E89C45F0FF
:1003640060305018E5825FFFE582F42B5582FB5024
:10037400210ABA001D09B90019088016E5825BFB41
:10038400E582F42F5582FF50090EBE00050DBD0015
:10039400010CC3EB9FF5F0EA9E42F0E99D42F0E8C0
:0D03A4009C45F06007CC4820E701B3EC2237
:1003B10075F020800E75F010800575F0087D007EC7
:1003C100007F003392D530D5031208D9EC334010A9
:1003D100EF33FFEE33FEED33FDEC33FCD5F0ED22D0
:0E03E100E5F0247EA2D513CC92E7CDCEFF220C
:1003EF00EDD2E7CD33EC3392D524814006E4FFFE06
:1003FF00FDFC22FCE4CFCECDCC24E0501174FF8065
:10040F00EDC3CC13CCCD13CDCE13CECF13CF047001
:07041F00F030D5DE0208D920
:10543400E55C2448F8E6055C227845301C0278488F
:10544400E475F001120A9C0207082015EB7F2ED2A6
:10545400158018EF540F2490D43440D4FF30190B26
:10546400EF24BFB41A0050032461FFE55D60021508
:105474005D0560E5607002055F301C0D7845E475DC
:10548400F001120A9CEF02074E02B3267403D21CE9
:105494008003E4C21CF55C8B458A468947E4F55DCC
:1054A400F55FF560E55D60077F2012546F80F57548
:1054B4005EFFC216C215C217C218C21AC21BC21D91
:1054C40012543DFF700D301C057F00125480AF60F4
:1054D400AE5F22B4255FC2D5C21912543DFF24D059
:1054E400B40A00501A75F00A785D30D50508B6FF85
:1054F4000106C6A426F620D5047002D21880D92449
:10550400CFB41A00EF5004C2E5D21902576DD21677
:1055140080C6D21580C0D21780BCD2D580BAD21A28
:1055240080B47F2012546F2017077401B55D0040CA
:10553400F1125434FF12546F0254A8D21DD21B80AE
:1055440095125434FB125434FA125434F94A4B7001
:105554000679647A587BFF20172EE55D602A7E0069
:105564008E8275830012072160060EEE655E70F070
:10557400C2D5EBC0E0EAC0E0E9C0E0EE1257CDD0FE
:10558400E0F9D0E0FAD0E0FB120708FF60AAEBC014
:10559400E0EAC0E0E9C0E012546FD0E02401F9D0A1
:1055A400E03400FAD0E0FBE55E0460DCD55ED9802F
:1055B40087D21780A21257B060F7E55E700104121B
:1055C4000470A95E600DE55E600914F55E1258571B
:1055D400EF60F3EA30E702F404C3995077EAF42564
:1055E4005E0430E701E404F55E800D1257B060C13B
:1055F400EA055E255E120470EA785BF630E701E4A2
:10560400255E04D55E04201A01141257CDE4C0E0CF
:10561400125857785BE6601320E70714F6125457C4
:10562400802204F6D0E014C0E07F00125457E55EF7
:10563400600712544E155E800B301A0312544ED07C
:10564400E00254A8D0E00480C51257B060A0E55E23
:1056540004120470785BEAF6E55E201A0260010425
:0556640024041257CDE3
:1056690074FF04C0E0125857125457E55E201A021D
:10567900600312544ED0E0B55EE87F45125461785C
:105689005BE67F2B30E7047F2DF404C0E012546FF2
:10569900D0E075F00A84C0F0125458D0E012545882
:1056A9000254A8791080027908C21BC21D8008D251
:1056B900D5790A8004790AC2D5E55E047002F55EDF
:1056C900E4FAFDFEFF125434FC7B08201613125431
:1056D90034FD7B1030150A125434FE125434FF7B0A
:1056E90020EC3382D592D55013C3E43015069FFFC1
:1056F900E49EFEE42016039DFDE49CFCE4CBF8C285
:1057090016EC700CCFCECDCCE824F8F870F38017E6
:10571900C3EF33FFEE33FEED33FDEC33FCEB33FB2C
:10572900994002FB0FD8E9EB301605F8D0E0C448E0
:10573900B216C0E00AEC4D4E4F78207B0070C2EAE9
:10574900B55E0040BCC0E01257CFD0F0D0E02016C3
:1057590004C4C0E0C4B216C0F0125458D0F0D5F059
:10576900EB0254A8120ADC55455356AC5855164C51
:1057790055124256B04F56B84456B849552B435660
:10578900BE5555EF46564D4555B947588450551A9B
:105799002D551E2E55412B552223553F20586D2A34
:1057A90054DA4800005539E55EB4FF03755E061208
:1057B9005434FC125434FD125434FE125434FF781C
:1057C9005402049F790AA2D5201814301A09B91075
:1057D900020404B9080104A2D5201B0250010420C7
:1057E90017689217B55D005034C0E07F2030181952
:1057F9007F30A217721B721A500F125826C217C295
:105809001BC21AC21D7F30800F301A03E9C0E01293
:10581900546F301A03D0E0F9D0E0B55DCC301A17D7
:105829007F30B9100C12546F7F583019077F788078
:1058390003B9080312546F3017057F2D02546F7F87
:1058490020201DF87F2B201BF322921780CF7F0089
:10585900B4070050052454F8E6FF22286E756C6CD5
:105869002900D2161254343016F8C216785D30D594
:105879000108F60254DA2D504349581254342403CE
:10588900B405004001E490587F93125460743A12B1
:0A5899005460D218755D040256AC8D
:0DB3C700ED33EC3360065004EC6480FC2292
:109C85008F478E468D458C4474FFFFFEFDFCAB4728
:109C9500AA46A945A844C31208FD602C7F807E967C
:109CA5007D187C4BAB47AA46A945A84412034460DE
:109CB5000250157F807E967D187CCBAB47AA46A9BE
:109CC50045A8441203445009AF47AE46AD45AC44E0
:109CD50022AF47AE46AD45AC441203EF8F4B8E4ADB
:109CE5008D498C48EC1203B1C8ECC8C9EDC9CAEE60
:109CF500CACBEFCBAF47AE46AD45AC441200A9E4A5
:109D0500FBFAF9F8120344601A401874FF254BF565
:109D15004BE54A34FFF54AE54934FFF549E5483452
:109D2500FFF548AF4BAE4AAD49AC48EC1203B12242
:10042600E9D2E7C933E833F892D5EDD2E7CD33EC1C
:0704360033FC5002B2D52295
:10043D00EC30E7100FBF000C0EBE00080DBD000420
:10044D000BEB6014A2D5EB13FCED92E7FD2274FFCC
:10045D00FCFDFEFF22E480F8A2D574FF13FC7D8025
:03046D00E480EF39
:10047000F920E72824F950037907E4F42402FB1853
:10048000DBFDE624FB5014E9600DE4F618E604F603
:0F049000B40A08E4F6D9F57401F60A22C2D5229F
:10049F00ED33EC3392D5FA602AB4FF33EDC2E77B2C
:1004AF00FF60067A0479C4E4227A0479CD20D5045A
:1004BF007A0479C8224E614E002B494E46002D49D1
:1004CF004E4600E47A08F608DAFC7B00740722E84F
:1004DF00C0E0ECC0E0EDC0E0EEC0E0EFC0E0EA75D8
:1004EF00F010A4CAABF075F04DA42BFBE435F0FC73
:1004FF00EA2410FAEB34C5FBEC34D9FCEDC2E7FF6C
:10050F0075F056A4F42411C5F0F434C58FF0A42A65
:10051F00E5F03BE43CF620E7141205D2D0E0FFD023
:10052F00E0FED0E0FDD0E0FC1202A78014F404122C
:10053F0005D2D0E0FFD0E0FED0E0FDD0E0FC12010C
:10054F009ED0E0F8E6FAEDD2E7CD33EC332482FB10
:10055F00E4C3CF33CFCE33CECD33CD33DBF37B07F5
:10056F0075F00A846004F6081B0AE5F0F6088FF0B0
:10057F00740AA4FFACF08EF0740AA42CFEACF050F9
:10058F00010C8DF0740AA42CFDE435F0F608DBDEC7
:03059F00740722BC
:1005A2003F8000004120000042C80000447A000061
:1005B200461C400047C35000497424004B189680E3
:1005C2004CBEBC205A0E1BCA6753C21C749DC5AEDA
:1005D200FB60065407601C2323120600EB543860AC
:1005E200091205EC1205FB12019EECF8EDF9EEFA88
:1005F200EFCB22EB1205FB80F1543803241C90054B
:10060200A2FE93FC0EEE93FD0EEE930ECE93FF220E
:0300000002A4490E
:0CA44900787FE4F6D8FD7581B102A49084
:10061200E709F608DFFA8046E709F208DFFA803ECA
:1006220088828C83E709F0A3DFFA8032E309F608B7
:10063200DFFA8078E309F208DFFA807088828C831F
:10064200E309F0A3DFFA806489828A83E0A3F608D3
:10065200DFFA805889828A83E0A3F208DFFA804CAD
:1006620080D280FA80C680D4806980F28033801084
:1006720080A680EA809A80A880DA80E280CA8033ED
:1006820089828A83ECFAE493A3C8C582C8CCC58365
:10069200CCF0A3C8C582C8CCC583CCDFE9DEE78035
:1006A2000D89828A83E493A3F608DFF9ECFAA9F0B4
:1006B200EDFB2289828A83ECFAE0A3C8C582C8CC0A
:1006C200C583CCF0A3C8C582C8CCC583CCDFEADE23
:1006D200E880DB89828A83E493A3F208DFF980CC85
:1006E20088F0EF60010E4E60C388F0ED2402B4047E
:1006F2000050B9F582EB2402B4040050AF23234525
:06070200822390066273E1
:10070800BB010689828A83E0225002E722BBFE02EF
:09071800E32289828A83E4932222
:10072100BB010CE58229F582E5833AF583E022508D
:1007310006E92582F8E622BBFE06E92582F8E222D7
:0D074100E58229F582E5833AF583E49322F1
:10074E00BB010689828A83F0225002F722BBFE018A
:02075E00F32284
:10076000F8BB010DE58229F582E5833AF583E8F0CF
:10077000225006E92582C8F622BBFE05E92582C87B
:02078000F22263
:10078200EF8DF0A4A8F0CF8CF0A428CE8DF0A42E8B
:02079200FE2245
:10079400BC000BBE0029EF8DF084FFADF022E4CC49
:1007A400F875F008EF2FFFEE33FEEC33FCEE9DEC12
:1007B400984005FCEE9DFE0FD5F0E9E4CEFD22ED58
:1007C400F8F5F0EE8420D21CFEADF075F008EF2FA2
:1007D400FFED33FD4007985006D5F0F222C398FD93
:0507E4000FD5F0EA2230
:1007E900C2D5EC30E709B2D5E4C39DFDE49CFCEE2B
:1007F90030E715B2D5E4C39FFFE49EFE120794C308
:10080900E49DFDE49CFC800312079430D507C3E402
:060819009FFFE49EFE2299
:10081F00BB010A89828A83E0F5F0A3E022500687A4
:10082F00F009E71922BBFE07E3F5F009E319228966
:0B083F00828A83E493F5F07401932299
:10084A00BB0110E58229F582E5833AF583E0F5F0EC
:10085A00A3E0225009E92582F886F008E622BBFEC9
:10086A000AE92582F8E2F5F008E222E5832AF5830F
:08087A00E993F5F0A3E99322D4
:10088200BB010789828A83020B5B500B09C5F027E3
:10089200F7C5F01937F722BBFE0D09F8E325F0F38F
:1008A200C5F019E338F322F889828A83740193250B
:0808B200F0C5F0F8E4933822D0
:1008BA00BB010A89828A83F0E5F0A3F0225006F789
:0F08CA0009A7F01922BBFE06F3E5F009F3192286
:0E08D900C3E49FFFE49EFEE49DFDE49CFC2230
:1008E700EB9FF5F0EA9E42F0E99D42F0EC6480C888
:0608F70064809845F02228
:1008FD00EB9FF5F0EA9E42F0E99D42F0E89C45F051
:01090D0022C7
:10090E00E8600FEFC333FFEE33FEED33FDEC33FC47
:03091E00D8F122EB
:10092100BB010789828A830209BB5005E9F80209E4
:10093100AFBBFE05E9F8020B7189828A83020B7D48
:10094100BB010DE58229F582E5833AF5830209BBF6
:100951005007E92582F80209AFBBFE07E92582F8B5
:10096100020B71E58229F582E5833AF583020B7D5D
:10097100BB010789828A83020A2C5005E9F8020A21
:0A09810020BBFE05E9F8020B9A22E4
:10098B00BB010DE58229F582E5833AF583020A2C3A
:10099B005007E92582F8020A20BBFE07E92582F8F9
:0409AB00020B9A227F
:0C09AF00E6FC08E6FD08E6FE08E6FF2274
:0C09BB00E0FCA3E0FDA3E0FEA3E0FF22AF
:0D09C700E6FB08E6F908E6FA08E6CBF822A0
:0C09D400E0F8A3E0F9A3E0FAA3E0FB22A6
:1009E000E493F8740193F9740293FA740393FB226D
:1009F000BB010DE58229F582E5833AF5830209D42E
:100A00005007E92582F80209C7BBFE07E92582F8ED
:100A1000020B8DE58229F582E5833AF5830209E030
:0C0A2000ECF608EDF608EEF608EFF62202
:0C0A2C00ECF0A3EDF0A3EEF0A3EFF0223D
:100A3800D083D082E493F608740193F60874029385
:090A4800F608740393F6740473BC
:100A5100A8828583F0D083D082120A68120A6812B4
:100A61000A68120A68E473E493A3C583C5F0C583D9
:100A7100C8C582C8F0A3C583C5F0C583C8C582C8EF
:010A81002252
:100A8200BB010789828A83020A515005E9F8020AEA
:0A0A920038BBFE05E9F8020BA622AE
:100A9C00FAE6FB0808E6F925F0F618E6CA3AF6225B
:100AAC00BB010DE58229F582E5833AF583020BC87B
:100ABC005007E92582F8020BBFBBFE07E92582F837
:100ACC00020BD1E58229F582E5833AF583020BDA34
:100ADC00D083D082F8E4937012740193700DA3A3A9
:100AEC0093F8740193F5828883E4737402936860BD
:060AFC00EFA3A3A380DFBD
:100B0200EC8EF0A4CCC5F0CCCDF8EFA4CEC5F02D80
:100B1200FDE43CFCE8A42EC8C5F03DFDE43CFCEF3E
:0D0B2200A4FFE5F028FEE43DFDE43CFC22CC
:10B12E00120708601CFF09E970010AC0E0EAC0E0DE
:10B13E00EBC0E012B326D0E0FBD0E0FAD0E0F9800D
:0AB14E00DF7F0A12B326E4FEFF22A1
:10AA84008B458A4689478B4B8A4C894DAB45054794
:10AA9400E547AA467002054614F912070870ED74DA
:10AAA400FF2547F54774FF3546F546AB48054AE5AB
:10AAB4004AAA497002054914F9120708FFAB450573
:10AAC40047E547AA467002054614F9EF12074E708F
:08AAD400DAAB4BAA4CA94D229C
:10ABDF008B458A468947E4F54DF54EE54C154CAE4D
:10ABEF004B7002154B4E6033AB48AA49A94A120766
:10ABFF0008FFAB45AA46A947054EE54EAC4D70027E
:10AC0F00054D14F5828C83EF120760EF60CD740150
:10AC1F00254AF54AE43549F54980C0AB45AA46A90E
:02AC2F004722BA
:10000E00E4FFFE120708600C0FEF70010E09E97095
:05001E00F20A80EF2250
:10B24200E94A4B700122120708FF6D700122EF706C
:0CB2520004FBFAF92209E970ED0A80EA19
:100B2F00EF4E6012EF60010EEDBB010B89828A83DD
:100B3F00F0A3DFFCDEFA2289F05007F709DFFCA9EA
:0C0B4F00F022BBFEFCF309DFFCA9F02241
:10A4550002B3ACE493A3F8E493A34003F68001F2BE
:10A4650008DFF48029E493A3F85407240CC8C33308
:10A47500C4540F4420C8834004F456800146F6DFD7
:10A48500E4800B010204081020408090ADBFE47EFB
:10A49500019360BCA3FF543F30E509541FFEE493CC
:10A4A500A360010ECF54C025E060A840B8E493A393
:10A4B500FAE493A3F8E493A3C8C582C8CAC583CABE
:10A4C500F0A3C8C582C8CAC583CADFE9DEE780BE76
:01AE0A000047
:100B5B00C5F0F8A3E028F0C5F0F8E5821582700225
:060B6B001583E038F022C2
:0C0B7100E2FC08E2FD08E2FE08E2FF22C0
:100B7D00E493FC740193FD740293FE740393FF22BE
:0D0B8D00E2FB08E2F908E2FA08E2CBF822E8
:0C0B9A00ECF208EDF208EEF208EFF22297
:100BA600D083D082E493F208740193F2087402931E
:090BB600F208740393F274047355
:090BBF00E6FB08E6FA08E6F9225B
:090BC800E0FBA3E0FAA3E0F9222E
:090BD100E2FB08E2FA08E2F92255
:0C0BDA00E493FB740193FA740293F92277
:00000001FF
